 zlib1

 Timestamp is 4f237e3a (Fri Jan 27 22:48:58 2012)

 Preferred load address is 10000000

 Start         Length     Name                   Class
 0001:00000000 00017f4aH .text                   CODE
 0002:00000000 00000110H .idata$5                DATA
 0002:00000110 00000004H .CRT$XCA                DATA
 0002:00000114 00000004H .CRT$XCZ                DATA
 0002:00000118 00000004H .CRT$XIA                DATA
 0002:0000011c 00000010H .CRT$XIC                DATA
 0002:0000012c 00000004H .CRT$XIZ                DATA
 0002:00000130 00000004H .CRT$XPA                DATA
 0002:00000134 00000004H .CRT$XPX                DATA
 0002:00000138 00000004H .CRT$XPXA               DATA
 0002:0000013c 00000004H .CRT$XPZ                DATA
 0002:00000140 00000004H .CRT$XTA                DATA
 0002:00000144 00000004H .CRT$XTZ                DATA
 0002:00000148 00005d98H .rdata                  DATA
 0002:00005ee0 00000004H .rtc$IAA                DATA
 0002:00005ee4 00000004H .rtc$IZZ                DATA
 0002:00005ee8 00000004H .rtc$TAA                DATA
 0002:00005eec 00000004H .rtc$TZZ                DATA
 0002:00005ef0 0000041cH .xdata$x                DATA
 0002:0000630c 00000014H .idata$2                DATA
 0002:00006320 00000014H .idata$3                DATA
 0002:00006334 00000110H .idata$4                DATA
 0002:00006444 000004caH .idata$6                DATA
 0002:00006910 00000c06H .edata                  DATA
 0003:00000000 00000facH .data                   DATA
 0003:00000fc0 00001ddcH .bss                    DATA
 0004:00000000 00000058H .rsrc$01                DATA
 0004:00000060 00000330H .rsrc$02                DATA

  Address         Publics by Value              Rva+Base       Lib:Object

 0000:00000000       __except_list              00000000     <absolute>
 0000:00000000       ___safe_se_handler_table   00000000     <absolute>
 0000:00000000       ___safe_se_handler_count   00000000     <absolute>
 0000:00000000       ___ImageBase               10000000     <linker-defined>
 0001:00000000       _adler32                   10001000 f   adler32.obj
 0001:00000310       _adler32_combine64         10001310 f   adler32.obj
 0001:00000310       _adler32_combine           10001310 f   adler32.obj
 0001:00000330       _compress2                 10001330 f   compress.obj
 0001:000003e0       _compress                  100013e0 f   compress.obj
 0001:00000400       _compressBound             10001400 f   compress.obj
 0001:00000420       _get_crc_table             10001420 f   crc32.obj
 0001:00000430       _crc32                     10001430 f   crc32.obj
 0001:00000820       _crc32_combine64           10001820 f   crc32.obj
 0001:00000820       _crc32_combine             10001820 f   crc32.obj
 0001:00000840       _deflateInit_              10001840 f   deflate.obj
 0001:00000870       _deflateInit2_             10001870 f   deflate.obj
 0001:00000ab0       _deflateSetDictionary      10001ab0 f   deflate.obj
 0001:00000bb0       _deflateReset              10001bb0 f   deflate.obj
 0001:00000c50       _deflateSetHeader          10001c50 f   deflate.obj
 0001:00000c80       _deflatePrime              10001c80 f   deflate.obj
 0001:00000cc0       _deflateParams             10001cc0 f   deflate.obj
 0001:00000dc0       _deflateTune               10001dc0 f   deflate.obj
 0001:00000e00       _deflateBound              10001e00 f   deflate.obj
 0001:00000f60       _deflate                   10001f60 f   deflate.obj
 0001:000017b0       _deflateEnd                100027b0 f   deflate.obj
 0001:00001890       _deflateCopy               10002890 f   deflate.obj
 0001:00002800       _gzclose                   10003800 f   gzclose.obj
 0001:00002a90       _gzopen                    10003a90 f   gzlib.obj
 0001:00002a90       _gzopen64                  10003a90 f   gzlib.obj
 0001:00002ab0       _gzdopen                   10003ab0 f   gzlib.obj
 0001:00002b00       _gzbuffer                  10003b00 f   gzlib.obj
 0001:00002b40       _gzrewind                  10003b40 f   gzlib.obj
 0001:00002b80       _gzseek64                  10003b80 f   gzlib.obj
 0001:00002ca0       _gzseek                    10003ca0 f   gzlib.obj
 0001:00002cb0       _gztell64                  10003cb0 f   gzlib.obj
 0001:00002cf0       _gztell                    10003cf0 f   gzlib.obj
 0001:00002d00       _gzoffset64                10003d00 f   gzlib.obj
 0001:00002d50       _gzoffset                  10003d50 f   gzlib.obj
 0001:00002d60       _gzeof                     10003d60 f   gzlib.obj
 0001:00002da0       _gzerror                   10003da0 f   gzlib.obj
 0001:00002de0       _gzclearerr                10003de0 f   gzlib.obj
 0001:00002e20       _gz_error                  10003e20 f   gzlib.obj
 0001:00003760       _gzread                    10004760 f   gzread.obj
 0001:000038c0       _gzgetc                    100048c0 f   gzread.obj
 0001:00003920       _gzungetc                  10004920 f   gzread.obj
 0001:000039f0       _gzgets                    100049f0 f   gzread.obj
 0001:00003af0       _gzdirect                  10004af0 f   gzread.obj
 0001:00003b20       _gzclose_r                 10004b20 f   gzread.obj
 0001:00003de0       _gzwrite                   10004de0 f   gzwrite.obj
 0001:00003ee0       _gzputc                    10004ee0 f   gzwrite.obj
 0001:00003f70       _gzputs                    10004f70 f   gzwrite.obj
 0001:00003fb0       _gzprintf                  10004fb0 f   gzwrite.obj
 0001:00004070       _gzflush                   10005070 f   gzwrite.obj
 0001:000040e0       _gzsetparams               100050e0 f   gzwrite.obj
 0001:00004180       _gzclose_w                 10005180 f   gzwrite.obj
 0001:00004210       _inflateBackInit_          10005210 f   infback.obj
 0001:000042f0       _inflateBack               100052f0 f   infback.obj
 0001:000050a0       _inflateBackEnd            100060a0 f   infback.obj
 0001:000050e0       _inflateReset              100060e0 f   inflate.obj
 0001:00005160       _inflateReset2             10006160 f   inflate.obj
 0001:000051f0       _inflateInit2_             100061f0 f   inflate.obj
 0001:000052b0       _inflateInit_              100062b0 f   inflate.obj
 0001:000052d0       _inflatePrime              100062d0 f   inflate.obj
 0001:00005450       _inflate                   10006450 f   inflate.obj
 0001:000069a0       _inflateEnd                100079a0 f   inflate.obj
 0001:000069f0       _inflateSetDictionary      100079f0 f   inflate.obj
 0001:00006ad0       _inflateGetHeader          10007ad0 f   inflate.obj
 0001:00006b60       _inflateSync               10007b60 f   inflate.obj
 0001:00006c40       _inflateSyncPoint          10007c40 f   inflate.obj
 0001:00006c70       _inflateCopy               10007c70 f   inflate.obj
 0001:00006dc0       _inflateUndermine          10007dc0 f   inflate.obj
 0001:00006df0       _inflateMark               10007df0 f   inflate.obj
 0001:00006e50       _inflate_table             10007e50 f   inftrees.obj
 0001:00007280       _call_zopen64              10008280 f   ioapi.obj
 0001:000072a0       _call_zseek64              100082a0 f   ioapi.obj
 0001:00007300       _call_ztell64              10008300 f   ioapi.obj
 0001:00007330       _fill_zlib_filefunc64_32_def_from_filefunc32 10008330 f   ioapi.obj
 0001:000074b0       _fill_fopen64_filefunc     100084b0 f   ioapi.obj
 0001:000075a0       _win32_open_file_func      100085a0 f   iowin32.obj
 0001:000075a0       _win32_open64_file_func    100085a0 f   iowin32.obj
 0001:000075a0       _win32_open64_file_funcA   100085a0 f   iowin32.obj
 0001:00007600       _win32_open64_file_funcW   10008600 f   iowin32.obj
 0001:00007660       _win32_read_file_func      10008660 f   iowin32.obj
 0001:000076b0       _win32_write_file_func     100086b0 f   iowin32.obj
 0001:00007700       _win32_tell_file_func      10008700 f   iowin32.obj
 0001:00007740       _win32_tell64_file_func    10008740 f   iowin32.obj
 0001:000077b0       _win32_seek_file_func      100087b0 f   iowin32.obj
 0001:00007810       _win32_seek64_file_func    10008810 f   iowin32.obj
 0001:00007870       _win32_close_file_func     10008870 f   iowin32.obj
 0001:000078a0       _win32_error_file_func     100088a0 f   iowin32.obj
 0001:000078c0       _fill_win32_filefunc       100088c0 f   iowin32.obj
 0001:00007900       _fill_win32_filefunc64A    10008900 f   iowin32.obj
 0001:00007900       _fill_win32_filefunc64     10008900 f   iowin32.obj
 0001:00007940       _fill_win32_filefunc64W    10008940 f   iowin32.obj
 0001:00007980       __tr_init                  10008980 f   trees.obj
 0001:00008920       __tr_stored_block          10009920 f   trees.obj
 0001:000089b0       __tr_align                 100099b0 f   trees.obj
 0001:00008ba0       __tr_flush_block           10009ba0 f   trees.obj
 0001:000093b0       _uncompress                1000a3b0 f   uncompr.obj
 0001:000096f0       _unzStringFileNameCompare  1000a6f0 f   unzip.obj
 0001:00009de0       _unzOpen2                  1000ade0 f   unzip.obj
 0001:00009e30       _unzOpen2_64               1000ae30 f   unzip.obj
 0001:00009e90       _unzOpen                   1000ae90 f   unzip.obj
 0001:00009eb0       _unzOpen64                 1000aeb0 f   unzip.obj
 0001:00009ed0       _unzClose                  1000aed0 f   unzip.obj
 0001:00009f10       _unzGetGlobalInfo64        1000af10 f   unzip.obj
 0001:00009f40       _unzGetGlobalInfo          1000af40 f   unzip.obj
 0001:0000a530       _unzGetCurrentFileInfo64   1000b530 f   unzip.obj
 0001:0000a560       _unzGetCurrentFileInfo     1000b560 f   unzip.obj
 0001:0000a630       _unzGoToFirstFile          1000b630 f   unzip.obj
 0001:0000a6a0       _unzGoToNextFile           1000b6a0 f   unzip.obj
 0001:0000a750       _unzLocateFile             1000b750 f   unzip.obj
 0001:0000a890       _unzGetFilePos64           1000b890 f   unzip.obj
 0001:0000a8e0       _unzGetFilePos             1000b8e0 f   unzip.obj
 0001:0000a910       _unzGoToFilePos64          1000b910 f   unzip.obj
 0001:0000a980       _unzGoToFilePos            1000b980 f   unzip.obj
 0001:0000ac00       _unzOpenCurrentFile3       1000bc00 f   unzip.obj
 0001:0000ae30       _unzOpenCurrentFile        1000be30 f   unzip.obj
 0001:0000ae50       _unzOpenCurrentFilePassword 1000be50 f   unzip.obj
 0001:0000ae70       _unzOpenCurrentFile2       1000be70 f   unzip.obj
 0001:0000ae90       _unzGetCurrentFileZStreamPos64 1000be90 f   unzip.obj
 0001:0000aec0       _unzReadCurrentFile        1000bec0 f   unzip.obj
 0001:0000b160       _unztell                   1000c160 f   unzip.obj
 0001:0000b180       _unztell64                 1000c180 f   unzip.obj
 0001:0000b1b0       _unzeof                    1000c1b0 f   unzip.obj
 0001:0000b1f0       _unzGetLocalExtrafield     1000c1f0 f   unzip.obj
 0001:0000b2b0       _unzCloseCurrentFile       1000c2b0 f   unzip.obj
 0001:0000b350       _unzGetGlobalComment       1000c350 f   unzip.obj
 0001:0000be50       _LoadCentralDirectoryRecord 1000ce50 f   zip.obj
 0001:0000c2f0       _zipOpen3                  1000d2f0 f   zip.obj
 0001:0000c450       _zipOpen2                  1000d450 f   zip.obj
 0001:0000c4a0       _zipOpen2_64               1000d4a0 f   zip.obj
 0001:0000c500       _zipOpen                   1000d500 f   zip.obj
 0001:0000c500       _zipOpen64                 1000d500 f   zip.obj
 0001:0000c520       _Write_LocalFileHeader     1000d520 f   zip.obj
 0001:0000c740       _zipOpenNewFileInZip4_64   1000d740 f   zip.obj
 0001:0000cc10       _zipOpenNewFileInZip3      1000dc10 f   zip.obj
 0001:0000cc70       _zipOpenNewFileInZip3_64   1000dc70 f   zip.obj
 0001:0000ccd0       _zipOpenNewFileInZip2      1000dcd0 f   zip.obj
 0001:0000cd20       _zipOpenNewFileInZip2_64   1000dd20 f   zip.obj
 0001:0000cd70       _zipOpenNewFileInZip64     1000dd70 f   zip.obj
 0001:0000cdc0       _zipOpenNewFileInZip       1000ddc0 f   zip.obj
 0001:0000ced0       _zipWriteInFileInZip       1000ded0 f   zip.obj
 0001:0000cfd0       _zipCloseFileInZipRaw      1000dfd0 f   zip.obj
 0001:0000cff0       _zipCloseFileInZipRaw64    1000dff0 f   zip.obj
 0001:0000d4e0       _zipCloseFileInZip         1000e4e0 f   zip.obj
 0001:0000d500       _Write_Zip64EndOfCentralDirectoryLocator 1000e500 f   zip.obj
 0001:0000d580       _Write_Zip64EndOfCentralDirectoryRecord 1000e580 f   zip.obj
 0001:0000d6a0       _Write_EndOfCentralDirectoryRecord 1000e6a0 f   zip.obj
 0001:0000d7e0       _Write_GlobalComment       1000e7e0 f   zip.obj
 0001:0000d850       _zipClose                  1000e850 f   zip.obj
 0001:0000d9c0       _zlibVersion               1000e9c0 f   zutil.obj
 0001:0000d9d0       _zlibCompileFlags          1000e9d0 f   zutil.obj
 0001:0000d9e0       _zError                    1000e9e0 f   zutil.obj
 0001:0000da00       _zcalloc                   1000ea00 f   zutil.obj
 0001:0000da20       _zcfree                    1000ea20 f   zutil.obj
 0001:0000da40       _longest_match             1000ea40 f   match686.obj
 0001:0000dc28       _match_init                1000ec28 f   match686.obj
 0001:0000dc30       _inflate_fast              1000ec30     inffas32.obj
 0001:0000e3cb       _sprintf                   1000f3cb f   LIBCMT:sprintf.obj
 0001:0000e44f       _free                      1000f44f f   LIBCMT:free.obj
 0001:0000e489       _malloc                    1000f489 f   LIBCMT:malloc.obj
 0001:0000e51d       __get_sys_err_msg          1000f51d f i LIBCMT:strerror.obj
 0001:0000e545       _strerror                  1000f545 f   LIBCMT:strerror.obj
 0001:0000e5b0       _memchr                    1000f5b0 f   LIBCMT:memchr.obj
 0001:0000e65d       __get_errno_from_oserr     1000f65d f   LIBCMT:dosmap.obj
 0001:0000e69f       __errno                    1000f69f f   LIBCMT:dosmap.obj
 0001:0000e6b2       ___doserrno                1000f6b2 f   LIBCMT:dosmap.obj
 0001:0000e6c5       __dosmaperr                1000f6c5 f   LIBCMT:dosmap.obj
 0001:0000e6e8       __vsnprintf_l              1000f6e8 f   LIBCMT:vsnprint.obj
 0001:0000e794       __vsnprintf                1000f794 f   LIBCMT:vsnprint.obj
 0001:0000e7b1       __ftelli64_nolock          1000f7b1 f   LIBCMT:ftelli64.obj
 0001:0000eafb       __ftelli64                 1000fafb f   LIBCMT:ftelli64.obj
 0001:0000eb68       __fseeki64_nolock          1000fb68 f   LIBCMT:fseeki64.obj
 0001:0000ec04       __fseeki64                 1000fc04 f   LIBCMT:fseeki64.obj
 0001:0000ec83       __fsopen                   1000fc83 f   LIBCMT:fopen.obj
 0001:0000ed3f       _fopen                     1000fd3f f   LIBCMT:fopen.obj
 0001:0000ed56       __fread_nolock_s           1000fd56 f   LIBCMT:fread.obj
 0001:0000ef12       _fread_s                   1000ff12 f   LIBCMT:fread.obj
 0001:0000efa0       _fread                     1000ffa0 f   LIBCMT:fread.obj
 0001:0000efbd       _ferror                    1000ffbd f   LIBCMT:feoferr.obj
 0001:0000efe5       __fwrite_nolock            1000ffe5 f   LIBCMT:fwrite.obj
 0001:0000f13c       _fwrite                    1001013c f   LIBCMT:fwrite.obj
 0001:0000f1b6       __fclose_nolock            100101b6 f   LIBCMT:fclose.obj
 0001:0000f223       _fclose                    10010223 f   LIBCMT:fclose.obj
 0001:0000f297       _srand                     10010297 f   LIBCMT:rand.obj
 0001:0000f2a9       _rand                      100102a9 f   LIBCMT:rand.obj
 0001:0000f2ca       __time64                   100102ca f   LIBCMT:time64.obj
 0001:0000f31b       __CRT_INIT@12              1001031b f   LIBCMT:dllcrt0.obj
 0001:0000f575       __DllMainCRTStartup@12     10010575 f   LIBCMT:dllcrt0.obj
 0001:0000f598       __flsbuf                   10010598 f   LIBCMT:_flsbuf.obj
 0001:0000f6fc       ??0_LocaleUpdate@@QAE@PAUlocaleinfo_struct@@@Z 100106fc f i LIBCMT:output.obj
 0001:0000f818       __output_l                 10010818 f   LIBCMT:output.obj
 0001:00010420       __initp_misc_invarg        10011420 f   LIBCMT:invarg.obj
 0001:0001042f       __call_reportfault         1001142f f   LIBCMT:invarg.obj
 0001:00010558       __invoke_watson            10011558 f   LIBCMT:invarg.obj
 0001:0001057d       __invalid_parameter        1001157d f   LIBCMT:invarg.obj
 0001:000105aa       __invalid_parameter_noinfo 100115aa f   LIBCMT:invarg.obj
 0001:000105ba       __heap_init                100115ba f   LIBCMT:heapinit.obj
 0001:000105d8       __heap_term                100115d8 f   LIBCMT:heapinit.obj
 0001:000105ec       ___crtCorExitProcess       100115ec f   LIBCMT:crt0dat.obj
 0001:00010617       ___crtExitProcess          10011617 f   LIBCMT:crt0dat.obj
 0001:0001062f       __lockexit                 1001162f f   LIBCMT:crt0dat.obj
 0001:00010638       __unlockexit               10011638 f   LIBCMT:crt0dat.obj
 0001:00010641       __init_pointers            10011641 f   LIBCMT:crt0dat.obj
 0001:00010674       __initterm_e               10011674 f   LIBCMT:crt0dat.obj
 0001:00010698       __cinit                    10011698 f   LIBCMT:crt0dat.obj
 0001:0001086f       __exit                     1001186f f   LIBCMT:crt0dat.obj
 0001:00010885       __cexit                    10011885 f   LIBCMT:crt0dat.obj
 0001:00010894       __amsg_exit                10011894 f   LIBCMT:crt0dat.obj
 0001:000108b2       __GET_RTERRMSG             100118b2 f   LIBCMT:crt0msg.obj
 0001:000108d8       __NMSG_WRITE               100118d8 f   LIBCMT:crt0msg.obj
 0001:00010a87       __FF_MSGBANNER             10011a87 f   LIBCMT:crt0msg.obj
 0001:00010ac0       __initp_heap_handler       10011ac0 f   LIBCMT:handler.obj
 0001:00010acf       __callnewh                 10011acf f   LIBCMT:handler.obj
 0001:00010af7       ___sys_nerr                10011af7 f   LIBCMT:syserr.obj
 0001:00010afd       ___sys_errlist             10011afd f   LIBCMT:syserr.obj
 0001:00010b03       _strcpy_s                  10011b03 f   LIBCMT:strcpy_s.obj
 0001:00010b62       __malloc_crt               10011b62 f   LIBCMT:crtheap.obj
 0001:00010ba7       __calloc_crt               10011ba7 f   LIBCMT:crtheap.obj
 0001:00010bf3       __realloc_crt              10011bf3 f   LIBCMT:crtheap.obj
 0001:00010c41       __encoded_null             10011c41 f   LIBCMT:tidtable.obj
 0001:00010c4a       ___crtTlsAlloc@4           10011c4a f   LIBCMT:tidtable.obj
 0001:00010c53       ___set_flsgetvalue         10011c53 f   LIBCMT:tidtable.obj
 0001:00010c87       __mtterm                   10011c87 f   LIBCMT:tidtable.obj
 0001:00010cc4       __initptd                  10011cc4 f   LIBCMT:tidtable.obj
 0001:00010d78       __getptd_noexit            10011d78 f   LIBCMT:tidtable.obj
 0001:00010df1       __getptd                   10011df1 f   LIBCMT:tidtable.obj
 0001:00010e0b       __freefls@4                10011e0b f   LIBCMT:tidtable.obj
 0001:00010f3a       __freeptd                  10011f3a f   LIBCMT:tidtable.obj
 0001:00010fa8       __mtinit                   10011fa8 f   LIBCMT:tidtable.obj
 0001:00011123       __read_nolock              10012123 f   LIBCMT:read.obj
 0001:000116da       __read                     100126da f   LIBCMT:read.obj
 0001:000116da       _read                      100126da f   LIBCMT:read.obj
 0001:000117d0       __ioinit                   100127d0 f   LIBCMT:ioinit.obj
 0001:00011a15       __ioterm                   10012a15 f   LIBCMT:ioinit.obj
 0001:00011a68       __lseeki64_nolock          10012a68 f   LIBCMT:lseeki64.obj
 0001:00011aed       __lseeki64                 10012aed f   LIBCMT:lseeki64.obj
 0001:00011bd7       __fileno                   10012bd7 f   LIBCMT:fileno.obj
 0001:00011bfd       @__security_check_cookie@4 10012bfd f   LIBCMT:secchk.obj
 0001:00011c10       __alloca_probe             10012c10     LIBCMT:chkstk.obj
 0001:00011c10       __chkstk                   10012c10 f   LIBCMT:chkstk.obj
 0001:00011c3b       ___iob_func                10012c3b f   LIBCMT:_file.obj
 0001:00011c41       ___initstdio               10012c41 f   LIBCMT:_file.obj
 0001:00011cf2       ___endstdio                10012cf2 f   LIBCMT:_file.obj
 0001:00011d12       __lock_file                10012d12 f   LIBCMT:_file.obj
 0001:00011d53       __lock_file2               10012d53 f   LIBCMT:_file.obj
 0001:00011d85       __unlock_file              10012d85 f   LIBCMT:_file.obj
 0001:00011dc1       __unlock_file2             10012dc1 f   LIBCMT:_file.obj
 0001:00011df0       __SEH_prolog4              10012df0 f   LIBCMT:sehprolg4.obj
 0001:00011e35       __SEH_epilog4              10012e35 f   LIBCMT:sehprolg4.obj
 0001:00011e50       __except_handler4          10012e50 f   LIBCMT:chandler4.obj
 0001:00011fdf       __flush                    10012fdf f   LIBCMT:fflush.obj
 0001:00012047       __fflush_nolock            10013047 f   LIBCMT:fflush.obj
 0001:00012169       __flushall                 10013169 f   LIBCMT:fflush.obj
 0001:00012172       __openfile                 10013172 f   LIBCMT:_open.obj
 0001:00012409       __getstream                10013409 f   LIBCMT:stream.obj
 0001:00012540       __local_unwind4            10013540 f   LIBCMT:exsup4.obj
 0001:00012616       __seh_longjmp_unwind4@4    10013616 f   LIBCMT:exsup4.obj
 0001:00012632       @_EH4_CallFilterFunc@8     10013632 f   LIBCMT:exsup4.obj
 0001:00012649       @_EH4_TransferToHandler@8  10013649 f   LIBCMT:exsup4.obj
 0001:00012662       @_EH4_GlobalUnwind2@8      10013662 f   LIBCMT:exsup4.obj
 0001:0001267b       @_EH4_LocalUnwind@16       1001367b f   LIBCMT:exsup4.obj
 0001:00012692       __filbuf                   10013692 f   LIBCMT:_filbuf.obj
 0001:000127b4       _memcpy_s                  100137b4 f   LIBCMT:memcpy_s.obj
 0001:00012830       _memset                    10013830 f   LIBCMT:memset.obj
 0001:000128aa       __write_nolock             100138aa f   LIBCMT:write.obj
 0001:00012fa7       __write                    10013fa7 f   LIBCMT:write.obj
 0001:00012fa7       _write                     10013fa7 f   LIBCMT:write.obj
 0001:00013080       _memcpy                    10014080 f   LIBCMT:memcpy.obj
 0001:000133e1       __lseek_nolock             100143e1 f   LIBCMT:lseek.obj
 0001:00013456       _lseek                     10014456 f   LIBCMT:lseek.obj
 0001:00013456       __lseek                    10014456 f   LIBCMT:lseek.obj
 0001:0001352a       __close_nolock             1001452a f   LIBCMT:close.obj
 0001:000135c6       _close                     100145c6 f   LIBCMT:close.obj
 0001:000135c6       __close                    100145c6 f   LIBCMT:close.obj
 0001:0001368a       __freebuf                  1001468a f   LIBCMT:_freebuf.obj
 0001:000136c0       __aulldiv                  100146c0 f   LIBCMT:ulldiv.obj
 0001:00013728       __setenvp                  10014728 f   LIBCMT:stdenvp.obj
 0001:0001399e       __setargv                  1001499e f   LIBCMT:stdargv.obj
 0001:00013a59       ___crtGetEnvironmentStringsA 10014a59 f   LIBCMT:a_env.obj
 0001:00013af0       __RTC_Initialize           10014af0 f   LIBCMT:_initsect_.obj
 0001:00013b16       __RTC_Terminate            10014b16 f   LIBCMT:_initsect_.obj
 0001:00013b3c       __XcptFilter               10014b3c f   LIBCMT:winxfltr.obj
 0001:00013c86       ___CppXcptFilter           10014c86 f   LIBCMT:winxfltr.obj
 0001:00013ca6       _DllMain@12                10014ca6 f   LIBCMT:dllmain.obj
 0001:00013cac       ___security_init_cookie    10014cac f   LIBCMT:gs_support.obj
 0001:00013d47       __getbuf                   10014d47 f   LIBCMT:_getbuf.obj
 0001:00013d90       __isatty                   10014d90 f   LIBCMT:isatty.obj
 0001:00014009       ___updatetmbcinfo          10015009 f   LIBCMT:mbctype.obj
 0001:00014129       __setmbcp_nolock           10015129 f   LIBCMT:mbctype.obj
 0001:00014312       __setmbcp                  10015312 f   LIBCMT:mbctype.obj
 0001:000144ac       ___initmbctable            100154ac f   LIBCMT:mbctype.obj
 0001:000144ca       ___addlocaleref            100154ca f   LIBCMT:localref.obj
 0001:00014559       ___removelocaleref         10015559 f   LIBCMT:localref.obj
 0001:000145f2       ___freetlocinfo            100155f2 f   LIBCMT:localref.obj
 0001:0001473d       __updatetlocinfoEx_nolock  1001573d f   LIBCMT:localref.obj
 0001:0001478a       ___updatetlocinfo          1001578a f   LIBCMT:localref.obj
 0001:00014803       __initp_misc_cfltcvt_tab   10015803 f   LIBCMT:cmiscdat.obj
 0001:00014826       __get_printf_count_output  10015826 f   LIBCMT:printf.obj
 0001:00014840       _strlen                    10015840 f   LIBCMT:strlen.obj
 0001:000148cb       __wctomb_s_l               100158cb f   LIBCMT:wctomb.obj
 0001:00014a20       _wctomb_s                  10015a20 f   LIBCMT:wctomb.obj
 0001:00014a3d       __isleadbyte_l             10015a3d f i LIBCMT:_wctype.obj
 0001:00014a75       _isleadbyte                10015a75 f i LIBCMT:_wctype.obj
 0001:00014a90       __aulldvrm                 10015a90 f   LIBCMT:ulldvrm.obj
 0001:00014b25       __crt_debugger_hook        10015b25 f   LIBCMT:dbghook.obj
 0001:00014b2d       __mtinitlocks              10015b2d f   LIBCMT:mlock.obj
 0001:00014b77       __mtdeletelocks            10015b77 f   LIBCMT:mlock.obj
 0001:00014bce       __unlock                   10015bce f   LIBCMT:mlock.obj
 0001:00014be5       __mtinitlocknum            10015be5 f   LIBCMT:mlock.obj
 0001:00014ca7       __lock                     10015ca7 f   LIBCMT:mlock.obj
 0001:00014cda       ?terminate@@YAXXZ          10015cda f   LIBCMT:hooks.obj
 0001:00014d13       __initp_eh_hooks           10015d13 f   LIBCMT:hooks.obj
 0001:00014d24       __initp_misc_winsig        10015d24 f   LIBCMT:winsig.obj
 0001:00014d79       ___get_sigabrt             10015d79 f   LIBCMT:winsig.obj
 0001:00014d86       _raise                     10015d86 f   LIBCMT:winsig.obj
 0001:00014f29       __initp_misc_rand_s        10015f29 f   LIBCMT:rand_s.obj
 0001:00014f38       __initp_misc_purevirt      10015f38 f   LIBCMT:inithelp.obj
 0001:00014ffd       ___onexitinit              10015ffd f   LIBCMT:onexit.obj
 0001:0001502e       __onexit                   1001602e f   LIBCMT:onexit.obj
 0001:0001506a       _atexit                    1001606a f   LIBCMT:onexit.obj
 0001:00015090       __ValidateImageBase        10016090 f   LIBCMT:pesect.obj
 0001:000150d0       __FindPESection            100160d0 f   LIBCMT:pesect.obj
 0001:00015120       __IsNonwritableInCurrentImage 10016120 f   LIBCMT:pesect.obj
 0001:000151dc       ___crtMessageBoxW          100161dc f   LIBCMT:crtmboxw.obj
 0001:00015348       _wcscat_s                  10016348 f   LIBCMT:wcscat_s.obj
 0001:000153bd       _wcsncpy_s                 100163bd f   LIBCMT:wcsncpy_s.obj
 0001:0001548a       _wcslen                    1001648a f   LIBCMT:wcslen.obj
 0001:000154a5       _wcscpy_s                  100164a5 f   LIBCMT:wcscpy_s.obj
 0001:00015508       __set_error_mode           10016508 f   LIBCMT:errmode.obj
 0001:00015547       __calloc_impl              10016547 f   LIBCMT:calloc_impl.obj
 0001:000155c9       _realloc                   100165c9 f   LIBCMT:realloc.obj
 0001:00015676       __set_osfhnd               10016676 f   LIBCMT:osfinfo.obj
 0001:000156f7       __free_osfhnd              100166f7 f   LIBCMT:osfinfo.obj
 0001:0001577d       __get_osfhandle            1001677d f   LIBCMT:osfinfo.obj
 0001:000157e6       ___lock_fhandle            100167e6 f   LIBCMT:osfinfo.obj
 0001:00015885       __unlock_fhandle           10016885 f   LIBCMT:osfinfo.obj
 0001:000158ac       __alloc_osfhnd             100168ac f   LIBCMT:osfinfo.obj
 0001:00015a45       ___report_gsfailure        10016a45 f   LIBCMT:gs_report.obj
 0001:00015b4b       __fcloseall                10016b4b f   LIBCMT:closeall.obj
 0001:00015be7       __commit                   10016be7 f   LIBCMT:commit.obj
 0001:000163f4       _open                      100173f4 f   LIBCMT:open.obj
 0001:000163f4       __open                     100173f4 f   LIBCMT:open.obj
 0001:000164a2       __sopen_helper             100174a2 f   LIBCMT:open.obj
 0001:00016566       __sopen_s                  10017566 f   LIBCMT:open.obj
 0001:00016586       __mbsnbicmp_l              10017586 f   LIBCMT:mbsnbicm.obj
 0001:0001678a       __mbsnbicmp                1001778a f   LIBCMT:mbsnbicm.obj
 0001:000167a4       __mbsnbcmp_l               100177a4 f   LIBCMT:mbsnbcmp.obj
 0001:000168f0       __mbsnbcmp                 100178f0 f   LIBCMT:mbsnbcmp.obj
 0001:00016910       __global_unwind2           10017910 f   LIBCMT:exsup.obj
 0001:00016975       __local_unwind2            10017975 f   LIBCMT:exsup.obj
 0001:000169f9       __abnormal_termination     100179f9 f   LIBCMT:exsup.obj
 0001:00016a1c       __NLG_Notify1              10017a1c f   LIBCMT:exsup.obj
 0001:00016a25       __NLG_Notify               10017a25 f   LIBCMT:exsup.obj
 0001:00016a3c       __NLG_Dispatch2            10017a3c     LIBCMT:exsup.obj
 0001:00016a3c       __NLG_Dispatch             10017a3c     LIBCMT:exsup.obj
 0001:00016a44       __NLG_Call                 10017a44 f   LIBCMT:exsup.obj
 0001:00016a46       __NLG_Return2              10017a46     LIBCMT:exsup.obj
 0001:00016a47       __VEC_memzero              10017a47 f   LIBCMT:p4_memset.obj
 0001:00016b01       ___sse2_available_init     10017b01 f   LIBCMT:cpu_disp.obj
 0001:00016b11       __putwch_nolock            10017b11 f   LIBCMT:putwch.obj
 0001:00016b53       __mbtowc_l                 10017b53 f   LIBCMT:mbtowc.obj
 0001:00016c69       _mbtowc                    10017c69 f   LIBCMT:mbtowc.obj
 0001:00016c83       __VEC_memcpy               10017c83 f   LIBCMT:p4_memcpy.obj
 0001:00016dd9       __ismbblead                10017dd9 f   LIBCMT:ismbbyte.obj
 0001:00016df1       __freea                    10017df1 f i LIBCMT:a_map.obj
 0001:00016ff8       ___crtLCMapStringA         10017ff8 f   LIBCMT:a_map.obj
 0001:00017125       ___crtGetStringTypeA       10018125 f   LIBCMT:a_str.obj
 0001:00017165       ___free_lc_time            10018165 f   LIBCMT:inittime.obj
 0001:000174dc       ___free_lconv_num          100184dc f   LIBCMT:initnum.obj
 0001:00017545       ___free_lconv_mon          10018545 f   LIBCMT:initmon.obj
 0001:00017643       __fptrap                   10018643 f   LIBCMT:crt0fp.obj
 0001:0001764c       _abort                     1001864c f   LIBCMT:abort.obj
 0001:0001767f       __msize                    1001867f f   LIBCMT:msize.obj
 0001:000176b2       __chsize_nolock            100186b2 f   LIBCMT:chsize.obj
 0001:00017868       __setmode_nolock           10018868 f   LIBCMT:setmode.obj
 0001:00017923       __get_fmode                10018923 f   LIBCMT:setmode.obj
 0001:00017950       __strnicmp_l               10018950 f   LIBCMT:strnicmp.obj
 0001:00017a32       __strnicmp                 10018a32 f   LIBCMT:strnicmp.obj
 0001:00017a85       _strncmp                   10018a85 f   LIBCMT:strncmp.obj
 0001:00017b45       ___initconout              10018b45 f   LIBCMT:initcon.obj
 0001:00017b64       ___termconout              10018b64 f   LIBCMT:initcon.obj
 0001:00017b80       __alloca_probe_16          10018b80 f   LIBCMT:alloca16.obj
 0001:00017b96       __alloca_probe_8           10018b96     LIBCMT:alloca16.obj
 0001:00017bac       __isctype_l                10018bac f   LIBCMT:isctype.obj
 0001:00017c64       __tolower_l                10018c64 f   LIBCMT:tolower.obj
 0001:00017d80       ___ascii_strnicmp          10018d80 f   LIBCMT:_strnicm.obj
 0001:00017df0       _strcspn                   10018df0 f   LIBCMT:strcspn.obj
 0001:00017e40       _strcmp                    10018e40 f   LIBCMT:strcmp.obj
 0001:00017ed0       _strpbrk                   10018ed0 f   LIBCMT:strpbrk.obj
 0001:00017f10       __allmul                   10018f10 f   LIBCMT:llmul.obj
 0001:00017f44       _RtlUnwind@16              10018f44 f   kernel32:KERNEL32.dll
 0002:00000000       __imp__CreateFileA@28      10019000     kernel32:KERNEL32.dll
 0002:00000004       __imp__SetFilePointer@16   10019004     kernel32:KERNEL32.dll
 0002:00000008       __imp__WriteFile@20        10019008     kernel32:KERNEL32.dll
 0002:0000000c       __imp__ReadFile@20         1001900c     kernel32:KERNEL32.dll
 0002:00000010       __imp__CreateFileW@28      10019010     kernel32:KERNEL32.dll
 0002:00000014       __imp__GetLastError@0      10019014     kernel32:KERNEL32.dll
 0002:00000018       __imp__CloseHandle@4       10019018     kernel32:KERNEL32.dll
 0002:0000001c       __imp__HeapFree@12         1001901c     kernel32:KERNEL32.dll
 0002:00000020       __imp__HeapAlloc@12        10019020     kernel32:KERNEL32.dll
 0002:00000024       __imp__GetSystemTimeAsFileTime@4 10019024     kernel32:KERNEL32.dll
 0002:00000028       __imp__GetCurrentThreadId@0 10019028     kernel32:KERNEL32.dll
 0002:0000002c       __imp__DecodePointer@4     1001902c     kernel32:KERNEL32.dll
 0002:00000030       __imp__GetCommandLineA@0   10019030     kernel32:KERNEL32.dll
 0002:00000034       __imp__UnhandledExceptionFilter@4 10019034     kernel32:KERNEL32.dll
 0002:00000038       __imp__SetUnhandledExceptionFilter@4 10019038     kernel32:KERNEL32.dll
 0002:0000003c       __imp__IsDebuggerPresent@0 1001903c     kernel32:KERNEL32.dll
 0002:00000040       __imp__EncodePointer@4     10019040     kernel32:KERNEL32.dll
 0002:00000044       __imp__TerminateProcess@8  10019044     kernel32:KERNEL32.dll
 0002:00000048       __imp__GetCurrentProcess@0 10019048     kernel32:KERNEL32.dll
 0002:0000004c       __imp__HeapCreate@12       1001904c     kernel32:KERNEL32.dll
 0002:00000050       __imp__HeapDestroy@4       10019050     kernel32:KERNEL32.dll
 0002:00000054       __imp__GetProcAddress@8    10019054     kernel32:KERNEL32.dll
 0002:00000058       __imp__GetModuleHandleW@4  10019058     kernel32:KERNEL32.dll
 0002:0000005c       __imp__ExitProcess@4       1001905c     kernel32:KERNEL32.dll
 0002:00000060       __imp__GetStdHandle@4      10019060     kernel32:KERNEL32.dll
 0002:00000064       __imp__GetModuleFileNameW@12 10019064     kernel32:KERNEL32.dll
 0002:00000068       __imp__Sleep@4             10019068     kernel32:KERNEL32.dll
 0002:0000006c       __imp__TlsAlloc@0          1001906c     kernel32:KERNEL32.dll
 0002:00000070       __imp__TlsGetValue@4       10019070     kernel32:KERNEL32.dll
 0002:00000074       __imp__TlsSetValue@8       10019074     kernel32:KERNEL32.dll
 0002:00000078       __imp__TlsFree@4           10019078     kernel32:KERNEL32.dll
 0002:0000007c       __imp__InterlockedIncrement@4 1001907c     kernel32:KERNEL32.dll
 0002:00000080       __imp__SetLastError@4      10019080     kernel32:KERNEL32.dll
 0002:00000084       __imp__InterlockedDecrement@4 10019084     kernel32:KERNEL32.dll
 0002:00000088       __imp__MultiByteToWideChar@24 10019088     kernel32:KERNEL32.dll
 0002:0000008c       __imp__SetHandleCount@4    1001908c     kernel32:KERNEL32.dll
 0002:00000090       __imp__InitializeCriticalSectionAndSpinCount@8 10019090     kernel32:KERNEL32.dll
 0002:00000094       __imp__GetFileType@4       10019094     kernel32:KERNEL32.dll
 0002:00000098       __imp__GetStartupInfoW@4   10019098     kernel32:KERNEL32.dll
 0002:0000009c       __imp__DeleteCriticalSection@4 1001909c     kernel32:KERNEL32.dll
 0002:000000a0       __imp__EnterCriticalSection@4 100190a0     kernel32:KERNEL32.dll
 0002:000000a4       __imp__LeaveCriticalSection@4 100190a4     kernel32:KERNEL32.dll
 0002:000000a8       __imp__RtlUnwind@16        100190a8     kernel32:KERNEL32.dll
 0002:000000ac       __imp__WideCharToMultiByte@32 100190ac     kernel32:KERNEL32.dll
 0002:000000b0       __imp__GetConsoleCP@0      100190b0     kernel32:KERNEL32.dll
 0002:000000b4       __imp__GetConsoleMode@8    100190b4     kernel32:KERNEL32.dll
 0002:000000b8       __imp__GetModuleFileNameA@12 100190b8     kernel32:KERNEL32.dll
 0002:000000bc       __imp__FreeEnvironmentStringsW@4 100190bc     kernel32:KERNEL32.dll
 0002:000000c0       __imp__GetEnvironmentStringsW@0 100190c0     kernel32:KERNEL32.dll
 0002:000000c4       __imp__QueryPerformanceCounter@4 100190c4     kernel32:KERNEL32.dll
 0002:000000c8       __imp__GetTickCount@0      100190c8     kernel32:KERNEL32.dll
 0002:000000cc       __imp__GetCurrentProcessId@0 100190cc     kernel32:KERNEL32.dll
 0002:000000d0       __imp__GetCPInfo@8         100190d0     kernel32:KERNEL32.dll
 0002:000000d4       __imp__GetACP@0            100190d4     kernel32:KERNEL32.dll
 0002:000000d8       __imp__GetOEMCP@0          100190d8     kernel32:KERNEL32.dll
 0002:000000dc       __imp__IsValidCodePage@4   100190dc     kernel32:KERNEL32.dll
 0002:000000e0       __imp__LoadLibraryW@4      100190e0     kernel32:KERNEL32.dll
 0002:000000e4       __imp__HeapReAlloc@16      100190e4     kernel32:KERNEL32.dll
 0002:000000e8       __imp__SetStdHandle@8      100190e8     kernel32:KERNEL32.dll
 0002:000000ec       __imp__FlushFileBuffers@4  100190ec     kernel32:KERNEL32.dll
 0002:000000f0       __imp__IsProcessorFeaturePresent@4 100190f0     kernel32:KERNEL32.dll
 0002:000000f4       __imp__WriteConsoleW@20    100190f4     kernel32:KERNEL32.dll
 0002:000000f8       __imp__LCMapStringW@24     100190f8     kernel32:KERNEL32.dll
 0002:000000fc       __imp__GetStringTypeW@16   100190fc     kernel32:KERNEL32.dll
 0002:00000100       __imp__HeapSize@12         10019100     kernel32:KERNEL32.dll
 0002:00000104       __imp__SetEndOfFile@4      10019104     kernel32:KERNEL32.dll
 0002:00000108       __imp__GetProcessHeap@0    10019108     kernel32:KERNEL32.dll
 0002:0000010c       \177KERNEL32_NULL_THUNK_DATA 1001910c     kernel32:KERNEL32.dll
 0002:00000110       ___xc_a                    10019110     LIBCMT:crt0init.obj
 0002:00000114       ___xc_z                    10019114     LIBCMT:crt0init.obj
 0002:00000118       ___xi_a                    10019118     LIBCMT:crt0init.obj
 0002:0000012c       ___xi_z                    1001912c     LIBCMT:crt0init.obj
 0002:00000130       ___xp_a                    10019130     LIBCMT:crt0init.obj
 0002:0000013c       ___xp_z                    1001913c     LIBCMT:crt0init.obj
 0002:00000140       ___xt_a                    10019140     LIBCMT:crt0init.obj
 0002:00000144       ___xt_z                    10019144     LIBCMT:crt0init.obj
 0002:00000148       ??_C@_0EA@FCLIIPNN@Visual?5C?$CL?$CL?5CRT?3?5Not?5enough?5memor@ 10019148     LIBCMT:strerror.obj
 0002:00000188       __pDefaultRawDllMain       10019188     LIBCMT:dllcrt0.obj
 0002:00000188       __pRawDllMain              10019188     LIBCMT:dllcrt0.obj
 0002:0000018c       ??_C@_1O@CEDCILHN@?$AA?$CI?$AAn?$AAu?$AAl?$AAl?$AA?$CJ?$AA?$AA@ 1001918c     LIBCMT:output.obj
 0002:0000019c       ??_C@_06OJHGLDPL@?$CInull?$CJ?$AA@ 1001919c     LIBCMT:output.obj
 0002:000001a8       ___lookuptable             100191a8     LIBCMT:output.obj
 0002:00000204       ??_C@_0P@MIGLKIOC@CorExitProcess?$AA@ 10019204     LIBCMT:crt0dat.obj
 0002:00000214       ??_C@_1BI@BGOHAHKC@?$AAm?$AAs?$AAc?$AAo?$AAr?$AAe?$AAe?$AA?4?$AAd?$AAl?$AAl?$AA?$AA@ 10019214     LIBCMT:crt0dat.obj
 0002:0000022c       ??_C@_1BO@BKOMIGKJ@?$AAr?$AAu?$AAn?$AAt?$AAi?$AAm?$AAe?$AA?5?$AAe?$AAr?$AAr?$AAo?$AAr?$AA?5?$AA?$AA@ 1001922c     LIBCMT:crt0msg.obj
 0002:0000024c       ??_C@_15JNBOKNOG@?$AA?$AN?$AA?6?$AA?$AA@ 1001924c     LIBCMT:crt0msg.obj
 0002:00000254       ??_C@_1BM@JBBEPPHI@?$AAT?$AAL?$AAO?$AAS?$AAS?$AA?5?$AAe?$AAr?$AAr?$AAo?$AAr?$AA?$AN?$AA?6?$AA?$AA@ 10019254     LIBCMT:crt0msg.obj
 0002:00000270       ??_C@_1BK@KMOMNAAI@?$AAS?$AAI?$AAN?$AAG?$AA?5?$AAe?$AAr?$AAr?$AAo?$AAr?$AA?$AN?$AA?6?$AA?$AA@ 10019270     LIBCMT:crt0msg.obj
 0002:0000028c       ??_C@_1BO@BFCDCGC@?$AAD?$AAO?$AAM?$AAA?$AAI?$AAN?$AA?5?$AAe?$AAr?$AAr?$AAo?$AAr?$AA?$AN?$AA?6?$AA?$AA@ 1001928c     LIBCMT:crt0msg.obj
 0002:000002b0       ??_C@_1BOO@KGEDBGAJ@?$AAR?$AA6?$AA0?$AA3?$AA3?$AA?$AN?$AA?6?$AA?9?$AA?5?$AAA?$AAt?$AAt?$AAe?$AAm?$AAp?$AAt?$AA?5?$AAt?$AAo?$AA?5?$AAu?$AAs?$AAe?$AA?5?$AAM?$AAS?$AAI?$AAL?$AA?5?$AAc?$AAo?$AAd@ 100192b0     LIBCMT:crt0msg.obj
 0002:000004a0       ??_C@_1GG@GOPILAJP@?$AAR?$AA6?$AA0?$AA3?$AA2?$AA?$AN?$AA?6?$AA?9?$AA?5?$AAn?$AAo?$AAt?$AA?5?$AAe?$AAn?$AAo?$AAu?$AAg?$AAh?$AA?5?$AAs?$AAp?$AAa?$AAc?$AAe?$AA?5?$AAf?$AAo?$AAr?$AA?5?$AAl?$AAo@ 100194a0     LIBCMT:crt0msg.obj
 0002:00000508       ??_C@_1MG@ENCOOIDF@?$AAR?$AA6?$AA0?$AA3?$AA1?$AA?$AN?$AA?6?$AA?9?$AA?5?$AAA?$AAt?$AAt?$AAe?$AAm?$AAp?$AAt?$AA?5?$AAt?$AAo?$AA?5?$AAi?$AAn?$AAi?$AAt?$AAi?$AAa?$AAl?$AAi?$AAz?$AAe?$AA?5?$AAt@ 10019508     LIBCMT:crt0msg.obj
 0002:000005d0       ??_C@_1DO@BMFCDCD@?$AAR?$AA6?$AA0?$AA3?$AA0?$AA?$AN?$AA?6?$AA?9?$AA?5?$AAC?$AAR?$AAT?$AA?5?$AAn?$AAo?$AAt?$AA?5?$AAi?$AAn?$AAi?$AAt?$AAi?$AAa?$AAl?$AAi?$AAz?$AAe?$AAd?$AA?$AN?$AA?6?$AA?$AA@ 100195d0     LIBCMT:crt0msg.obj
 0002:00000610       ??_C@_1EK@HHFLMAOL@?$AAR?$AA6?$AA0?$AA2?$AA8?$AA?$AN?$AA?6?$AA?9?$AA?5?$AAu?$AAn?$AAa?$AAb?$AAl?$AAe?$AA?5?$AAt?$AAo?$AA?5?$AAi?$AAn?$AAi?$AAt?$AAi?$AAa?$AAl?$AAi?$AAz?$AAe?$AA?5?$AAh?$AAe@ 10019610     LIBCMT:crt0msg.obj
 0002:00000660       ??_C@_1GK@MFGOKLAG@?$AAR?$AA6?$AA0?$AA2?$AA7?$AA?$AN?$AA?6?$AA?9?$AA?5?$AAn?$AAo?$AAt?$AA?5?$AAe?$AAn?$AAo?$AAu?$AAg?$AAh?$AA?5?$AAs?$AAp?$AAa?$AAc?$AAe?$AA?5?$AAf?$AAo?$AAr?$AA?5?$AAl?$AAo@ 10019660     LIBCMT:crt0msg.obj
 0002:000006d0       ??_C@_1GK@MCAAGJMO@?$AAR?$AA6?$AA0?$AA2?$AA6?$AA?$AN?$AA?6?$AA?9?$AA?5?$AAn?$AAo?$AAt?$AA?5?$AAe?$AAn?$AAo?$AAu?$AAg?$AAh?$AA?5?$AAs?$AAp?$AAa?$AAc?$AAe?$AA?5?$AAf?$AAo?$AAr?$AA?5?$AAs?$AAt@ 100196d0     LIBCMT:crt0msg.obj
 0002:00000740       ??_C@_1EM@MAADIHMB@?$AAR?$AA6?$AA0?$AA2?$AA5?$AA?$AN?$AA?6?$AA?9?$AA?5?$AAp?$AAu?$AAr?$AAe?$AA?5?$AAv?$AAi?$AAr?$AAt?$AAu?$AAa?$AAl?$AA?5?$AAf?$AAu?$AAn?$AAc?$AAt?$AAi?$AAo?$AAn?$AA?5?$AAc@ 10019740     LIBCMT:crt0msg.obj
 0002:00000790       ??_C@_1GK@FHCKBEFA@?$AAR?$AA6?$AA0?$AA2?$AA4?$AA?$AN?$AA?6?$AA?9?$AA?5?$AAn?$AAo?$AAt?$AA?5?$AAe?$AAn?$AAo?$AAu?$AAg?$AAh?$AA?5?$AAs?$AAp?$AAa?$AAc?$AAe?$AA?5?$AAf?$AAo?$AAr?$AA?5?$AA_?$AAo@ 10019790     LIBCMT:crt0msg.obj
 0002:00000800       ??_C@_1FC@ECHBIFBC@?$AAR?$AA6?$AA0?$AA1?$AA9?$AA?$AN?$AA?6?$AA?9?$AA?5?$AAu?$AAn?$AAa?$AAb?$AAl?$AAe?$AA?5?$AAt?$AAo?$AA?5?$AAo?$AAp?$AAe?$AAn?$AA?5?$AAc?$AAo?$AAn?$AAs?$AAo?$AAl?$AAe?$AA?5@ 10019800     LIBCMT:crt0msg.obj
 0002:00000858       ??_C@_1EC@JIBHAOPH@?$AAR?$AA6?$AA0?$AA1?$AA8?$AA?$AN?$AA?6?$AA?9?$AA?5?$AAu?$AAn?$AAe?$AAx?$AAp?$AAe?$AAc?$AAt?$AAe?$AAd?$AA?5?$AAh?$AAe?$AAa?$AAp?$AA?5?$AAe?$AAr?$AAr?$AAo?$AAr?$AA?$AN?$AA?6@ 10019858     LIBCMT:crt0msg.obj
 0002:000008a0       ??_C@_1FK@BEOGODMC@?$AAR?$AA6?$AA0?$AA1?$AA7?$AA?$AN?$AA?6?$AA?9?$AA?5?$AAu?$AAn?$AAe?$AAx?$AAp?$AAe?$AAc?$AAt?$AAe?$AAd?$AA?5?$AAm?$AAu?$AAl?$AAt?$AAi?$AAt?$AAh?$AAr?$AAe?$AAa?$AAd?$AA?5@ 100198a0     LIBCMT:crt0msg.obj
 0002:00000900       ??_C@_1FI@LOGNIKDM@?$AAR?$AA6?$AA0?$AA1?$AA6?$AA?$AN?$AA?6?$AA?9?$AA?5?$AAn?$AAo?$AAt?$AA?5?$AAe?$AAn?$AAo?$AAu?$AAg?$AAh?$AA?5?$AAs?$AAp?$AAa?$AAc?$AAe?$AA?5?$AAf?$AAo?$AAr?$AA?5?$AAt?$AAh@ 10019900     LIBCMT:crt0msg.obj
 0002:00000958       ??_C@_1EG@BEHAGFJD@?$AAR?$AA6?$AA0?$AA1?$AA0?$AA?$AN?$AA?6?$AA?9?$AA?5?$AAa?$AAb?$AAo?$AAr?$AAt?$AA?$CI?$AA?$CJ?$AA?5?$AAh?$AAa?$AAs?$AA?5?$AAb?$AAe?$AAe?$AAn?$AA?5?$AAc?$AAa?$AAl?$AAl?$AAe?$AAd@ 10019958     LIBCMT:crt0msg.obj
 0002:000009a0       ??_C@_1FI@HONFMGBI@?$AAR?$AA6?$AA0?$AA0?$AA9?$AA?$AN?$AA?6?$AA?9?$AA?5?$AAn?$AAo?$AAt?$AA?5?$AAe?$AAn?$AAo?$AAu?$AAg?$AAh?$AA?5?$AAs?$AAp?$AAa?$AAc?$AAe?$AA?5?$AAf?$AAo?$AAr?$AA?5?$AAe?$AAn@ 100199a0     LIBCMT:crt0msg.obj
 0002:000009f8       ??_C@_1FE@LLNEDJMD@?$AAR?$AA6?$AA0?$AA0?$AA8?$AA?$AN?$AA?6?$AA?9?$AA?5?$AAn?$AAo?$AAt?$AA?5?$AAe?$AAn?$AAo?$AAu?$AAg?$AAh?$AA?5?$AAs?$AAp?$AAa?$AAc?$AAe?$AA?5?$AAf?$AAo?$AAr?$AA?5?$AAa?$AAr@ 100199f8     LIBCMT:crt0msg.obj
 0002:00000a50       ??_C@_1FK@PGACCAFB@?$AAR?$AA6?$AA0?$AA0?$AA2?$AA?$AN?$AA?6?$AA?9?$AA?5?$AAf?$AAl?$AAo?$AAa?$AAt?$AAi?$AAn?$AAg?$AA?5?$AAp?$AAo?$AAi?$AAn?$AAt?$AA?5?$AAs?$AAu?$AAp?$AAp?$AAo?$AAr?$AAt?$AA?5@ 10019a50     LIBCMT:crt0msg.obj
 0002:00000b60       ??_C@_1EK@MBDPDCGA@?$AAM?$AAi?$AAc?$AAr?$AAo?$AAs?$AAo?$AAf?$AAt?$AA?5?$AAV?$AAi?$AAs?$AAu?$AAa?$AAl?$AA?5?$AAC?$AA?$CL?$AA?$CL?$AA?5?$AAR?$AAu?$AAn?$AAt?$AAi?$AAm?$AAe?$AA?5?$AAL?$AAi?$AAb@ 10019b60     LIBCMT:crt0msg.obj
 0002:00000bac       ??_C@_15IABLJNFO@?$AA?6?$AA?6?$AA?$AA@ 10019bac     LIBCMT:crt0msg.obj
 0002:00000bb4       ??_C@_17LGKOMLJ@?$AA?4?$AA?4?$AA?4?$AA?$AA@ 10019bb4     LIBCMT:crt0msg.obj
 0002:00000bbc       ??_C@_1CO@EAEJAADC@?$AA?$DM?$AAp?$AAr?$AAo?$AAg?$AAr?$AAa?$AAm?$AA?5?$AAn?$AAa?$AAm?$AAe?$AA?5?$AAu?$AAn?$AAk?$AAn?$AAo?$AAw?$AAn?$AA?$DO?$AA?$AA@ 10019bbc     LIBCMT:crt0msg.obj
 0002:00000bec       ??_C@_1DE@JNGNBFGO@?$AAR?$AAu?$AAn?$AAt?$AAi?$AAm?$AAe?$AA?5?$AAE?$AAr?$AAr?$AAo?$AAr?$AA?$CB?$AA?6?$AA?6?$AAP?$AAr?$AAo?$AAg?$AAr?$AAa?$AAm?$AA?3?$AA?5?$AA?$AA@ 10019bec     LIBCMT:crt0msg.obj
 0002:00000c20       ??_C@_0BG@KLEAJEFJ@Illegal?5byte?5sequence?$AA@ 10019c20     LIBCMT:syserr.obj
 0002:00000c38       ??_C@_0BE@ICMCHPHH@Directory?5not?5empty?$AA@ 10019c38     LIBCMT:syserr.obj
 0002:00000c4c       ??_C@_0BJ@IHEHINLI@Function?5not?5implemented?$AA@ 10019c4c     LIBCMT:syserr.obj
 0002:00000c68       ??_C@_0BD@CLHBCGPB@No?5locks?5available?$AA@ 10019c68     LIBCMT:syserr.obj
 0002:00000c7c       ??_C@_0BC@BEDIHIDK@Filename?5too?5long?$AA@ 10019c7c     LIBCMT:syserr.obj
 0002:00000c90       ??_C@_0BK@JAEBMJJM@Resource?5deadlock?5avoided?$AA@ 10019c90     LIBCMT:syserr.obj
 0002:00000cac       ??_C@_0BB@FCBJFCAJ@Result?5too?5large?$AA@ 10019cac     LIBCMT:syserr.obj
 0002:00000cc0       ??_C@_0N@MMJPGLJK@Domain?5error?$AA@ 10019cc0     LIBCMT:syserr.obj
 0002:00000cd0       ??_C@_0M@LHEPIIOM@Broken?5pipe?$AA@ 10019cd0     LIBCMT:syserr.obj
 0002:00000cdc       ??_C@_0P@PKCJJLLM@Too?5many?5links?$AA@ 10019cdc     LIBCMT:syserr.obj
 0002:00000cec       ??_C@_0BG@DDBFNKBH@Read?9only?5file?5system?$AA@ 10019cec     LIBCMT:syserr.obj
 0002:00000d04       ??_C@_0N@FEHLOILP@Invalid?5seek?$AA@ 10019d04     LIBCMT:syserr.obj
 0002:00000d14       ??_C@_0BI@FEALHKLD@No?5space?5left?5on?5device?$AA@ 10019d14     LIBCMT:syserr.obj
 0002:00000d2c       ??_C@_0P@LFMMIPAE@File?5too?5large?$AA@ 10019d2c     LIBCMT:syserr.obj
 0002:00000d3c       ??_C@_0CE@ONOKNLPF@Inappropriate?5I?1O?5control?5operat@ 10019d3c     LIBCMT:syserr.obj
 0002:00000d60       ??_C@_0BE@INBJMKGG@Too?5many?5open?5files?$AA@ 10019d60     LIBCMT:syserr.obj
 0002:00000d74       ??_C@_0BO@IIFBODJE@Too?5many?5open?5files?5in?5system?$AA@ 10019d74     LIBCMT:syserr.obj
 0002:00000d94       ??_C@_0BB@HMGGCEBG@Invalid?5argument?$AA@ 10019d94     LIBCMT:syserr.obj
 0002:00000da8       ??_C@_0P@NDHGCGKE@Is?5a?5directory?$AA@ 10019da8     LIBCMT:syserr.obj
 0002:00000db8       ??_C@_0BA@CJBACOOL@Not?5a?5directory?$AA@ 10019db8     LIBCMT:syserr.obj
 0002:00000dc8       ??_C@_0P@NLEIANHE@No?5such?5device?$AA@ 10019dc8     LIBCMT:syserr.obj
 0002:00000dd8       ??_C@_0O@OAMDNOCP@Improper?5link?$AA@ 10019dd8     LIBCMT:syserr.obj
 0002:00000de8       ??_C@_0M@NAAJNNGH@File?5exists?$AA@ 10019de8     LIBCMT:syserr.obj
 0002:00000df4       ??_C@_0BA@BIBLIOEK@Resource?5device?$AA@ 10019df4     LIBCMT:syserr.obj
 0002:00000e04       ??_C@_0O@NIPGCINC@Unknown?5error?$AA@ 10019e04     LIBCMT:syserr.obj
 0002:00000e14       ??_C@_0M@LOEHLCJD@Bad?5address?$AA@ 10019e14     LIBCMT:syserr.obj
 0002:00000e20       ??_C@_0BC@HFNFNKAI@Permission?5denied?$AA@ 10019e20     LIBCMT:syserr.obj
 0002:00000e34       ??_C@_0BB@IMDKMPFB@Not?5enough?5space?$AA@ 10019e34     LIBCMT:syserr.obj
 0002:00000e48       ??_C@_0CB@EPFKGNAK@Resource?5temporarily?5unavailable@ 10019e48     LIBCMT:syserr.obj
 0002:00000e6c       ??_C@_0BD@LOHELEP@No?5child?5processes?$AA@ 10019e6c     LIBCMT:syserr.obj
 0002:00000e80       ??_C@_0BE@NFGDDCEF@Bad?5file?5descriptor?$AA@ 10019e80     LIBCMT:syserr.obj
 0002:00000e94       ??_C@_0BC@HKPNECK@Exec?5format?5error?$AA@ 10019e94     LIBCMT:syserr.obj
 0002:00000ea8       ??_C@_0BC@MFFGCDFL@Arg?5list?5too?5long?$AA@ 10019ea8     LIBCMT:syserr.obj
 0002:00000ebc       ??_C@_0BK@DPKMCKJ@No?5such?5device?5or?5address?$AA@ 10019ebc     LIBCMT:syserr.obj
 0002:00000ed8       ??_C@_0BD@KKNFOBBD@Input?1output?5error?$AA@ 10019ed8     LIBCMT:syserr.obj
 0002:00000eec       ??_C@_0BK@FJBOAFDK@Interrupted?5function?5call?$AA@ 10019eec     LIBCMT:syserr.obj
 0002:00000f08       ??_C@_0BA@FKIAIBGA@No?5such?5process?$AA@ 10019f08     LIBCMT:syserr.obj
 0002:00000f18       ??_C@_0BK@FMDHKPNF@No?5such?5file?5or?5directory?$AA@ 10019f18     LIBCMT:syserr.obj
 0002:00000f34       ??_C@_0BI@BJFCGOHL@Operation?5not?5permitted?$AA@ 10019f34     LIBCMT:syserr.obj
 0002:00000f4c       ??_C@_08INEPGKHH@No?5error?$AA@ 10019f4c     LIBCMT:syserr.obj
 0002:00000f58       ??_C@_1BK@DBDEIDLH@?$AAK?$AAE?$AAR?$AAN?$AAE?$AAL?$AA3?$AA2?$AA?4?$AAD?$AAL?$AAL?$AA?$AA@ 10019f58     LIBCMT:tidtable.obj
 0002:00000f74       ??_C@_07PEJMOBNF@FlsFree?$AA@ 10019f74     LIBCMT:tidtable.obj
 0002:00000f7c       ??_C@_0M@JCPCPOEF@FlsSetValue?$AA@ 10019f7c     LIBCMT:tidtable.obj
 0002:00000f88       ??_C@_0M@GDNOONDI@FlsGetValue?$AA@ 10019f88     LIBCMT:tidtable.obj
 0002:00000f94       ??_C@_08KNHFBNJ@FlsAlloc?$AA@ 10019f94     LIBCMT:tidtable.obj
 0002:00000fc0       __XcptActTab               10019fc0     LIBCMT:winxfltr.obj
 0002:00001050       __First_FPE_Indx           1001a050     LIBCMT:winxfltr.obj
 0002:00001054       __Num_FPE                  1001a054     LIBCMT:winxfltr.obj
 0002:00001058       __XcptActTabSize           1001a058     LIBCMT:winxfltr.obj
 0002:0000105c       __XcptActTabCount          1001a05c     LIBCMT:winxfltr.obj
 0002:00001060       ??_C@_1BC@GDGBMEMK@?$AAH?$AAH?$AA?3?$AAm?$AAm?$AA?3?$AAs?$AAs?$AA?$AA@ 1001a060     LIBCMT:nlsdata2.obj
 0002:00001074       ??_C@_1CI@KNAKOEBC@?$AAd?$AAd?$AAd?$AAd?$AA?0?$AA?5?$AAM?$AAM?$AAM?$AAM?$AA?5?$AAd?$AAd?$AA?0?$AA?5?$AAy?$AAy?$AAy?$AAy?$AA?$AA@ 1001a074     LIBCMT:nlsdata2.obj
 0002:0000109c       ??_C@_1BC@IEBCMHCM@?$AAM?$AAM?$AA?1?$AAd?$AAd?$AA?1?$AAy?$AAy?$AA?$AA@ 1001a09c     LIBCMT:nlsdata2.obj
 0002:000010b0       ??_C@_15CLMNNGEL@?$AAP?$AAM?$AA?$AA@ 1001a0b0     LIBCMT:nlsdata2.obj
 0002:000010b8       ??_C@_15ODEHAHHF@?$AAA?$AAM?$AA?$AA@ 1001a0b8     LIBCMT:nlsdata2.obj
 0002:000010c0       ??_C@_1BC@FEMKIFH@?$AAD?$AAe?$AAc?$AAe?$AAm?$AAb?$AAe?$AAr?$AA?$AA@ 1001a0c0     LIBCMT:nlsdata2.obj
 0002:000010d4       ??_C@_1BC@BGLIFPF@?$AAN?$AAo?$AAv?$AAe?$AAm?$AAb?$AAe?$AAr?$AA?$AA@ 1001a0d4     LIBCMT:nlsdata2.obj
 0002:000010e8       ??_C@_1BA@EPANDLNG@?$AAO?$AAc?$AAt?$AAo?$AAb?$AAe?$AAr?$AA?$AA@ 1001a0e8     LIBCMT:nlsdata2.obj
 0002:000010f8       ??_C@_1BE@DKAAMBJL@?$AAS?$AAe?$AAp?$AAt?$AAe?$AAm?$AAb?$AAe?$AAr?$AA?$AA@ 1001a0f8     LIBCMT:nlsdata2.obj
 0002:0000110c       ??_C@_1O@PAHLKOAC@?$AAA?$AAu?$AAg?$AAu?$AAs?$AAt?$AA?$AA@ 1001a10c     LIBCMT:nlsdata2.obj
 0002:0000111c       ??_C@_19BIFMLPCD@?$AAJ?$AAu?$AAl?$AAy?$AA?$AA@ 1001a11c     LIBCMT:nlsdata2.obj
 0002:00001128       ??_C@_19EPFLPGAP@?$AAJ?$AAu?$AAn?$AAe?$AA?$AA@ 1001a128     LIBCMT:nlsdata2.obj
 0002:00001134       ??_C@_1M@GJNLMHFD@?$AAA?$AAp?$AAr?$AAi?$AAl?$AA?$AA@ 1001a134     LIBCMT:nlsdata2.obj
 0002:00001140       ??_C@_1M@IKEENEDF@?$AAM?$AAa?$AAr?$AAc?$AAh?$AA?$AA@ 1001a140     LIBCMT:nlsdata2.obj
 0002:0000114c       ??_C@_1BC@JGDDFFAM@?$AAF?$AAe?$AAb?$AAr?$AAu?$AAa?$AAr?$AAy?$AA?$AA@ 1001a14c     LIBCMT:nlsdata2.obj
 0002:00001160       ??_C@_1BA@EFMEIEBA@?$AAJ?$AAa?$AAn?$AAu?$AAa?$AAr?$AAy?$AA?$AA@ 1001a160     LIBCMT:nlsdata2.obj
 0002:00001170       ??_C@_17EGKACKIF@?$AAD?$AAe?$AAc?$AA?$AA@ 1001a170     LIBCMT:nlsdata2.obj
 0002:00001178       ??_C@_17BBDMLCIG@?$AAN?$AAo?$AAv?$AA?$AA@ 1001a178     LIBCMT:nlsdata2.obj
 0002:00001180       ??_C@_17FNLKOI@?$AAO?$AAc?$AAt?$AA?$AA@ 1001a180     LIBCMT:nlsdata2.obj
 0002:00001188       ??_C@_17HCHCOKMG@?$AAS?$AAe?$AAp?$AA?$AA@ 1001a188     LIBCMT:nlsdata2.obj
 0002:00001190       ??_C@_17ICPELBCN@?$AAA?$AAu?$AAg?$AA?$AA@ 1001a190     LIBCMT:nlsdata2.obj
 0002:00001198       ??_C@_17IJPCKHK@?$AAJ?$AAu?$AAl?$AA?$AA@ 1001a198     LIBCMT:nlsdata2.obj
 0002:000011a0       ??_C@_17KCJGOCPB@?$AAJ?$AAu?$AAn?$AA?$AA@ 1001a1a0     LIBCMT:nlsdata2.obj
 0002:000011a8       ??_C@_17PNNKMEED@?$AAM?$AAa?$AAy?$AA?$AA@ 1001a1a8     LIBCMT:nlsdata2.obj
 0002:000011b0       ??_C@_17LFPOIHDD@?$AAA?$AAp?$AAr?$AA?$AA@ 1001a1b0     LIBCMT:nlsdata2.obj
 0002:000011b8       ??_C@_17CKNLEDEC@?$AAM?$AAa?$AAr?$AA?$AA@ 1001a1b8     LIBCMT:nlsdata2.obj
 0002:000011c0       ??_C@_17LMDJEKJN@?$AAF?$AAe?$AAb?$AA?$AA@ 1001a1c0     LIBCMT:nlsdata2.obj
 0002:000011c8       ??_C@_17DKNBKCHM@?$AAJ?$AAa?$AAn?$AA?$AA@ 1001a1c8     LIBCMT:nlsdata2.obj
 0002:000011d0       ??_C@_1BC@ENMNNPAJ@?$AAS?$AAa?$AAt?$AAu?$AAr?$AAd?$AAa?$AAy?$AA?$AA@ 1001a1d0     LIBCMT:nlsdata2.obj
 0002:000011e4       ??_C@_1O@PDICJHAG@?$AAF?$AAr?$AAi?$AAd?$AAa?$AAy?$AA?$AA@ 1001a1e4     LIBCMT:nlsdata2.obj
 0002:000011f4       ??_C@_1BC@HHMNLIHE@?$AAT?$AAh?$AAu?$AAr?$AAs?$AAd?$AAa?$AAy?$AA?$AA@ 1001a1f4     LIBCMT:nlsdata2.obj
 0002:00001208       ??_C@_1BE@EBOGMDOH@?$AAW?$AAe?$AAd?$AAn?$AAe?$AAs?$AAd?$AAa?$AAy?$AA?$AA@ 1001a208     LIBCMT:nlsdata2.obj
 0002:0000121c       ??_C@_1BA@ENFBFFEK@?$AAT?$AAu?$AAe?$AAs?$AAd?$AAa?$AAy?$AA?$AA@ 1001a21c     LIBCMT:nlsdata2.obj
 0002:0000122c       ??_C@_1O@MMNBFLIA@?$AAM?$AAo?$AAn?$AAd?$AAa?$AAy?$AA?$AA@ 1001a22c     LIBCMT:nlsdata2.obj
 0002:0000123c       ??_C@_1O@IHNHDHPB@?$AAS?$AAu?$AAn?$AAd?$AAa?$AAy?$AA?$AA@ 1001a23c     LIBCMT:nlsdata2.obj
 0002:0000124c       ??_C@_17GGIBDPIH@?$AAS?$AAa?$AAt?$AA?$AA@ 1001a24c     LIBCMT:nlsdata2.obj
 0002:00001254       ??_C@_17HFOLPPLP@?$AAF?$AAr?$AAi?$AA?$AA@ 1001a254     LIBCMT:nlsdata2.obj
 0002:0000125c       ??_C@_17PDPHAADD@?$AAT?$AAh?$AAu?$AA?$AA@ 1001a25c     LIBCMT:nlsdata2.obj
 0002:00001264       ??_C@_17CJEDCEPE@?$AAW?$AAe?$AAd?$AA?$AA@ 1001a264     LIBCMT:nlsdata2.obj
 0002:0000126c       ??_C@_17BMKGEGOJ@?$AAT?$AAu?$AAe?$AA?$AA@ 1001a26c     LIBCMT:nlsdata2.obj
 0002:00001274       ??_C@_17KBOMKBF@?$AAM?$AAo?$AAn?$AA?$AA@ 1001a274     LIBCMT:nlsdata2.obj
 0002:0000127c       ??_C@_17MBGCMIPB@?$AAS?$AAu?$AAn?$AA?$AA@ 1001a27c     LIBCMT:nlsdata2.obj
 0002:00001284       ??_C@_08JCCMCCIL@HH?3mm?3ss?$AA@ 1001a284     LIBCMT:nlsdata2.obj
 0002:00001290       ??_C@_0BE@CKGJFCPC@dddd?0?5MMMM?5dd?0?5yyyy?$AA@ 1001a290     LIBCMT:nlsdata2.obj
 0002:000012a4       ??_C@_08BPBNCDIB@MM?1dd?1yy?$AA@ 1001a2a4     LIBCMT:nlsdata2.obj
 0002:000012b0       ??_C@_02CJNFDJBF@PM?$AA@   1001a2b0     LIBCMT:nlsdata2.obj
 0002:000012b4       ??_C@_02DEDBPAFC@AM?$AA@   1001a2b4     LIBCMT:nlsdata2.obj
 0002:000012b8       ??_C@_08EDHMEBNP@December?$AA@ 1001a2b8     LIBCMT:nlsdata2.obj
 0002:000012c4       ??_C@_08HCHEGEOA@November?$AA@ 1001a2c4     LIBCMT:nlsdata2.obj
 0002:000012d0       ??_C@_07JJNFCEND@October?$AA@ 1001a2d0     LIBCMT:nlsdata2.obj
 0002:000012d8       ??_C@_09BHHEALKD@September?$AA@ 1001a2d8     LIBCMT:nlsdata2.obj
 0002:000012e4       ??_C@_06LBBHFDDG@August?$AA@ 1001a2e4     LIBCMT:nlsdata2.obj
 0002:000012ec       ??_C@_04MIEPOIFP@July?$AA@ 1001a2ec     LIBCMT:nlsdata2.obj
 0002:000012f4       ??_C@_04CNLMGBGM@June?$AA@ 1001a2f4     LIBCMT:nlsdata2.obj
 0002:000012fc       ??_C@_05DMJDNLEJ@April?$AA@ 1001a2fc     LIBCMT:nlsdata2.obj
 0002:00001304       ??_C@_05HPCKOFNC@March?$AA@ 1001a304     LIBCMT:nlsdata2.obj
 0002:0000130c       ??_C@_08GNJGEPFN@February?$AA@ 1001a30c     LIBCMT:nlsdata2.obj
 0002:00001318       ??_C@_07CGJPFGJA@January?$AA@ 1001a318     LIBCMT:nlsdata2.obj
 0002:00001320       ??_C@_03MKABNOCG@Dec?$AA@  1001a320     LIBCMT:nlsdata2.obj
 0002:00001324       ??_C@_03JPJOFNIA@Nov?$AA@  1001a324     LIBCMT:nlsdata2.obj
 0002:00001328       ??_C@_03BMAOKBAD@Oct?$AA@  1001a328     LIBCMT:nlsdata2.obj
 0002:0000132c       ??_C@_03GGCAPAJC@Sep?$AA@  1001a32c     LIBCMT:nlsdata2.obj
 0002:00001330       ??_C@_03IFJFEIGA@Aug?$AA@  1001a330     LIBCMT:nlsdata2.obj
 0002:00001334       ??_C@_03LBGABGKK@Jul?$AA@  1001a334     LIBCMT:nlsdata2.obj
 0002:00001338       ??_C@_03IDFGHECI@Jun?$AA@  1001a338     LIBCMT:nlsdata2.obj
 0002:0000133c       ??_C@_03CNMDKL@May?$AA@    1001a33c     LIBCMT:nlsdata2.obj
 0002:00001340       ??_C@_03LEOLGMJP@Apr?$AA@  1001a340     LIBCMT:nlsdata2.obj
 0002:00001344       ??_C@_03ODNJBKGA@Mar?$AA@  1001a344     LIBCMT:nlsdata2.obj
 0002:00001348       ??_C@_03HJBDCHOM@Feb?$AA@  1001a348     LIBCMT:nlsdata2.obj
 0002:0000134c       ??_C@_03JIHJHPIE@Jan?$AA@  1001a34c     LIBCMT:nlsdata2.obj
 0002:00001350       ??_C@_08INBOOONO@Saturday?$AA@ 1001a350     LIBCMT:nlsdata2.obj
 0002:0000135c       ??_C@_06JECMNKMI@Friday?$AA@ 1001a35c     LIBCMT:nlsdata2.obj
 0002:00001364       ??_C@_08HACCIKIA@Thursday?$AA@ 1001a364     LIBCMT:nlsdata2.obj
 0002:00001370       ??_C@_09DLIGFAKA@Wednesday?$AA@ 1001a370     LIBCMT:nlsdata2.obj
 0002:0000137c       ??_C@_07BAAGCFCM@Tuesday?$AA@ 1001a37c     LIBCMT:nlsdata2.obj
 0002:00001384       ??_C@_06JLEDEDGH@Monday?$AA@ 1001a384     LIBCMT:nlsdata2.obj
 0002:0000138c       ??_C@_06OOPIFAJ@Sunday?$AA@ 1001a38c     LIBCMT:nlsdata2.obj
 0002:00001394       ??_C@_03FEFJNEK@Sat?$AA@   1001a394     LIBCMT:nlsdata2.obj
 0002:00001398       ??_C@_03IDIOELNC@Fri?$AA@  1001a398     LIBCMT:nlsdata2.obj
 0002:0000139c       ??_C@_03IOFIKPDN@Thu?$AA@  1001a39c     LIBCMT:nlsdata2.obj
 0002:000013a0       ??_C@_03MHOMLAJA@Wed?$AA@  1001a3a0     LIBCMT:nlsdata2.obj
 0002:000013a4       ??_C@_03NAGEINEP@Tue?$AA@  1001a3a4     LIBCMT:nlsdata2.obj
 0002:000013a8       ??_C@_03PDAGKDH@Mon?$AA@   1001a3a8     LIBCMT:nlsdata2.obj
 0002:000013ac       ??_C@_03KOEHGMDN@Sun?$AA@  1001a3ac     LIBCMT:nlsdata2.obj
 0002:000013b0       ___lookuptable_s           1001a3b0     LIBCMT:outputs.obj
 0002:0000140c       ??_C@_0BI@DFKBFLJE@GetProcessWindowStation?$AA@ 1001a40c     LIBCMT:crtmboxw.obj
 0002:00001424       ??_C@_0BK@DEKFELLI@GetUserObjectInformationW?$AA@ 1001a424     LIBCMT:crtmboxw.obj
 0002:00001440       ??_C@_0BD@HHGDFDBJ@GetLastActivePopup?$AA@ 1001a440     LIBCMT:crtmboxw.obj
 0002:00001454       ??_C@_0BA@HNOPNCHB@GetActiveWindow?$AA@ 1001a454     LIBCMT:crtmboxw.obj
 0002:00001464       ??_C@_0M@DLDCCGNP@MessageBoxW?$AA@ 1001a464     LIBCMT:crtmboxw.obj
 0002:00001470       ??_C@_1BG@GOEBHBDC@?$AAU?$AAS?$AAE?$AAR?$AA3?$AA2?$AA?4?$AAD?$AAL?$AAL?$AA?$AA@ 1001a470     LIBCMT:crtmboxw.obj
 0002:00001490       ___newctype                1001a490     LIBCMT:ctype.obj
 0002:00001790       __wctype                   1001a790     LIBCMT:ctype.obj
 0002:00001998       ___newclmap                1001a998     LIBCMT:ctype.obj
 0002:00001b18       ___newcumap                1001ab18     LIBCMT:ctype.obj
 0002:00001c98       ??_C@_1BA@BALFACEM@?$AAC?$AAO?$AAN?$AAO?$AAU?$AAT?$AA$?$AA?$AA@ 1001ac98     LIBCMT:initcon.obj
 0002:00001d28       ??_C@_05DFCKICEH@1?42?45?$AA@ 1001ad28     compress.obj
 0002:00001d30       _z_errmsg                  1001ad30     zutil.obj
 0002:00001d58       _zip_copyright             1001ad58     zip.obj
 0002:00001da8       _unz_copyright             1001ada8     unzip.obj
 0002:00002448       __dist_code                1001b448     trees.obj
 0002:00002648       __length_code              1001b648     trees.obj
 0002:00002838       _inflate_copyright         1001b838     inftrees.obj
 0002:00003ab8       _deflate_copyright         1001cab8     deflate.obj
 0002:00005b80       ??_C@_07EBNKNFJN@?$DMfd?3?$CFd?$DO?$AA@ 1001eb80     gzlib.obj
 0002:00005b88       ??_C@_00CNPNBAHC@?$AA@     1001eb88     gzlib.obj
 0002:00005b8c       ??_C@_0O@BNNCBLEN@out?5of?5memory?$AA@ 1001eb8c     gzlib.obj
 0002:00005b9c       ??_C@_02LMMGGCAJ@?3?5?$AA@ 1001eb9c     gzlib.obj
 0002:00005ba0       ??_C@_0BL@IHKGDAEE@unknown?5compression?5method?$AA@ 1001eba0     gzread.obj
 0002:00005bbc       ??_C@_0BJ@BLBBCOMO@unknown?5header?5flags?5set?$AA@ 1001ebbc     gzread.obj
 0002:00005bd8       ??_C@_0BH@CFIIDOJD@unexpected?5end?5of?5file?$AA@ 1001ebd8     gzread.obj
 0002:00005bf0       ??_C@_0CH@CPOLIEKA@internal?5error?3?5inflate?5stream?5c@ 1001ebf0     gzread.obj
 0002:00005c18       ??_C@_0BG@HCKBMIHF@compressed?5data?5error?$AA@ 1001ec18     gzread.obj
 0002:00005c30       ??_C@_0BF@MEIGEHBE@incorrect?5data?5check?$AA@ 1001ec30     gzread.obj
 0002:00005c48       ??_C@_0BH@FGKKJGOC@incorrect?5length?5check?$AA@ 1001ec48     gzread.obj
 0002:00005c60       ??_C@_0CF@MLPJFDMM@requested?5length?5does?5not?5fit?5in@ 1001ec60     gzread.obj
 0002:00005c88       ??_C@_0BP@IIKIGMCC@out?5of?5room?5to?5push?5characters?$AA@ 1001ec88     gzread.obj
 0002:00005ca8       ??_C@_0CH@DEEGAHIB@internal?5error?3?5deflate?5stream?5c@ 1001eca8     gzwrite.obj
 0002:00005cd0       ??_C@_0BD@PJCBIDD@invalid?5block?5type?$AA@ 1001ecd0     infback.obj
 0002:00005ce4       ??_C@_0BN@LGAADGOK@invalid?5stored?5block?5lengths?$AA@ 1001ece4     infback.obj
 0002:00005d04       ??_C@_0CE@GMIGFPBB@too?5many?5length?5or?5distance?5symb@ 1001ed04     infback.obj
 0002:00005d28       ??_C@_0BJ@HDEPPGOH@invalid?5code?5lengths?5set?$AA@ 1001ed28     infback.obj
 0002:00005d44       ??_C@_0BK@BMMPFBBH@invalid?5bit?5length?5repeat?$AA@ 1001ed44     infback.obj
 0002:00005d60       ??_C@_0CF@DGDMADCD@invalid?5code?5?9?9?5missing?5end?9of?9b@ 1001ed60     infback.obj
 0002:00005d88       ??_C@_0BM@IIMGAINC@invalid?5literal?1lengths?5set?$AA@ 1001ed88     infback.obj
 0002:00005da4       ??_C@_0BG@GMDFCBGP@invalid?5distances?5set?$AA@ 1001eda4     infback.obj
 0002:00005dbc       ??_C@_0BM@FFFLPBBC@invalid?5literal?1length?5code?$AA@ 1001edbc     infback.obj
 0002:00005dd8       ??_C@_0BG@LBKINIKP@invalid?5distance?5code?$AA@ 1001edd8     infback.obj
 0002:00005df0       ??_C@_0BO@ECPMAOGG@invalid?5distance?5too?5far?5back?$AA@ 1001edf0     infback.obj
 0002:00005e10       ??_C@_0BH@LIBMMIGA@incorrect?5header?5check?$AA@ 1001ee10     inflate.obj
 0002:00005e28       ??_C@_0BE@EMOGCLGO@invalid?5window?5size?$AA@ 1001ee28     inflate.obj
 0002:00005e3c       ??_C@_0BE@GONKLEPM@header?5crc?5mismatch?$AA@ 1001ee3c     inflate.obj
 0002:00005e50       ??_C@_02JDPG@rb?$AA@       1001ee50     ioapi.obj
 0002:00005e54       ??_C@_03HMFOOINA@r?$CLb?$AA@ 1001ee54     ioapi.obj
 0002:00005e58       ??_C@_02GMLFBBN@wb?$AA@    1001ee58     ioapi.obj
 0002:00005e5c       ??_C@_01JOAMLHOP@?9?$AA@   1001ee5c     zip.obj
 0002:00005e60       ??_C@_0BF@CJFPCCEG@incompatible?5version?$AA@ 1001ee60     zutil.obj
 0002:00005e78       ??_C@_0N@DFPGLBGC@buffer?5error?$AA@ 1001ee78     zutil.obj
 0002:00005e88       ??_C@_0BE@OGGJBMCE@insufficient?5memory?$AA@ 1001ee88     zutil.obj
 0002:00005e9c       ??_C@_0L@HAHMBNLP@data?5error?$AA@ 1001ee9c     zutil.obj
 0002:00005ea8       ??_C@_0N@MKKNPMJD@stream?5error?$AA@ 1001eea8     zutil.obj
 0002:00005eb8       ??_C@_0L@KIJFAKBJ@file?5error?$AA@ 1001eeb8     zutil.obj
 0002:00005ec4       ??_C@_0L@FNAOCBOG@stream?5end?$AA@ 1001eec4     zutil.obj
 0002:00005ed0       ??_C@_0BA@MOKMMFOD@need?5dictionary?$AA@ 1001eed0     zutil.obj
 0002:00005ee0       ___rtc_iaa                 1001eee0     LIBCMT:_initsect_.obj
 0002:00005ee4       ___rtc_izz                 1001eee4     LIBCMT:_initsect_.obj
 0002:00005ee8       ___rtc_taa                 1001eee8     LIBCMT:_initsect_.obj
 0002:00005eec       ___rtc_tzz                 1001eeec     LIBCMT:_initsect_.obj
 0002:0000630c       __IMPORT_DESCRIPTOR_KERNEL32 1001f30c     kernel32:KERNEL32.dll
 0002:00006320       __NULL_IMPORT_DESCRIPTOR   1001f320     kernel32:KERNEL32.dll
 0003:00000180       ___nullstring              10021180     LIBCMT:output.obj
 0003:00000184       ___wnullstring             10021184     LIBCMT:output.obj
 0003:00000188       __sys_errlist              10021188     LIBCMT:syserr.obj
 0003:00000238       __sys_nerr                 10021238     LIBCMT:syserr.obj
 0003:0000023c       ___flsindex                1002123c     LIBCMT:tidtable.obj
 0003:00000240       ___getvalueindex           10021240     LIBCMT:tidtable.obj
 0003:00000248       __lookuptrailbytes         10021248     LIBCMT:read.obj
 0003:00000348       ___badioinfo               10021348     LIBCMT:ioinit.obj
 0003:00000388       ___security_cookie         10021388     LIBCMT:gs_cookie.obj
 0003:0000038c       ___security_cookie_complement 1002138c     LIBCMT:gs_cookie.obj
 0003:00000390       __iob                      10021390     LIBCMT:_file.obj
 0003:00000610       ___initialmbcinfo          10021610     LIBCMT:mbctype.obj
 0003:00000830       __mbctype                  10021830     LIBCMT:mbctype.obj
 0003:00000938       __mbcasemap                10021938     LIBCMT:mbctype.obj
 0003:00000a38       ___ptmbcinfo               10021a38     LIBCMT:mbctype.obj
 0003:00000b30       ___globallocalestatus      10021b30     LIBCMT:glstatus.obj
 0003:00000b34       ___clocalestr              10021b34     LIBCMT:nlsdata2.obj
 0003:00000b38       ___lc_time_c               10021b38     LIBCMT:nlsdata2.obj
 0003:00000ca0       ___initiallocinfo          10021ca0     LIBCMT:nlsdata2.obj
 0003:00000d78       ___ptlocinfo               10021d78     LIBCMT:nlsdata2.obj
 0003:00000d7c       __cfltcvt_tab              10021d7c     LIBCMT:cmiscdat.obj
 0003:00000ed0       __NLG_Destination          10021ed0     LIBCMT:exsup.obj
 0003:00000ee0       ___lconv_static_decimal    10021ee0     LIBCMT:lconv.obj
 0003:00000ee4       ___lconv_static_W_decimal  10021ee4     LIBCMT:lconv.obj
 0003:00000ee8       ___lconv_c                 10021ee8     LIBCMT:lconv.obj
 0003:00000f38       ___lconv                   10021f38     LIBCMT:lconv.obj
 0003:00000f3c       __pctype                   10021f3c     LIBCMT:ctype.obj
 0003:00000f40       __pwctype                  10021f40     LIBCMT:ctype.obj
 0003:00000f44       ___abort_behavior          10021f44     LIBCMT:abort.obj
 0003:00000f48       __confh                    10021f48     LIBCMT:initcon.obj
 0003:00000f60       ___mb_cur_max              10021f60     LIBCMT:nlsdata1.obj
 0003:00000f64       ___decimal_point           10021f64     LIBCMT:nlsdata1.obj
 0003:00000f68       ___decimal_point_length    10021f68     LIBCMT:nlsdata1.obj
 0003:00000fc4       __aenvptr                  10021fc4     LIBCMT:dllcrt0.obj
 0003:00000fc8       __wenvptr                  10021fc8     LIBCMT:dllcrt0.obj
 0003:00000fcc       ___error_mode              10021fcc     LIBCMT:dllcrt0.obj
 0003:00000fd0       ___app_type                10021fd0     LIBCMT:dllcrt0.obj
 0003:00000fd4       ___pInvalidArgHandler      10021fd4     LIBCMT:invarg.obj
 0003:00000fd8       __crtheap                  10021fd8     LIBCMT:heapinit.obj
 0003:00000fdc       __umaskval                 10021fdc     LIBCMT:crt0dat.obj
 0003:00000fe0       ___argc                    10021fe0     LIBCMT:crt0dat.obj
 0003:00000fe4       ___argv                    10021fe4     LIBCMT:crt0dat.obj
 0003:00000fe8       ___wargv                   10021fe8     LIBCMT:crt0dat.obj
 0003:00000fec       __environ                  10021fec     LIBCMT:crt0dat.obj
 0003:00000ff0       ___initenv                 10021ff0     LIBCMT:crt0dat.obj
 0003:00000ff4       __wenviron                 10021ff4     LIBCMT:crt0dat.obj
 0003:00000ff8       ___winitenv                10021ff8     LIBCMT:crt0dat.obj
 0003:00000ffc       __pgmptr                   10021ffc     LIBCMT:crt0dat.obj
 0003:00001000       __wpgmptr                  10022000     LIBCMT:crt0dat.obj
 0003:00001004       __exitflag                 10022004     LIBCMT:crt0dat.obj
 0003:00001008       __C_Termination_Done       10022008     LIBCMT:crt0dat.obj
 0003:0000100c       __C_Exit_Done              1002200c     LIBCMT:crt0dat.obj
 0003:00001638       ?_pnhHeap@@3P6AHI@ZA       10022638     LIBCMT:handler.obj
 0003:0000163c       __newmode                  1002263c     LIBCMT:_newmode.obj
 0003:00001640       __maxwait                  10022640     LIBCMT:crtheap.obj
 0003:00001644       _gpFlsAlloc                10022644     LIBCMT:tidtable.obj
 0003:00001648       _gpFlsGetValue             10022648     LIBCMT:tidtable.obj
 0003:0000164c       _gpFlsSetValue             1002264c     LIBCMT:tidtable.obj
 0003:00001650       _gpFlsFree                 10022650     LIBCMT:tidtable.obj
 0003:00001654       __cflush                   10022654     LIBCMT:_file.obj
 0003:00001764       ___mbulinfo                10022764     LIBCMT:mbctype.obj
 0003:00001770       ___mbcodepage              10022770     LIBCMT:mbctype.obj
 0003:00001774       ___ismbcodepage            10022774     LIBCMT:mbctype.obj
 0003:00001778       ___mblcid                  10022778     LIBCMT:mbctype.obj
 0003:000018d0       ?__pInconsistency@@3P6AXXZA 100228d0     LIBCMT:hooks.obj
 0003:000018ec       ___pPurecall               100228ec     LIBCMT:inithelp.obj
 0003:00001c2c       __commode                  10022c2c     LIBCMT:ncommode.obj
 0003:00001c30       ___lconv_static_null       10022c30     LIBCMT:lconv.obj
 0003:00001c34       ___lconv_static_W_null     10022c34     LIBCMT:lconv.obj
 0003:00001c38       __stdbuf                   10022c38     LIBCMT:_sftbuf.obj
 0003:00001c40       ___locale_changed          10022c40     LIBCMT:setlocal.obj
 0003:00001c44       __fmode                    10022c44     LIBCMT:txtmode.obj
 0003:00001c4c       ___sse2_available          10022c4c     <common>
 0003:00001c50       __debugger_hook_dummy      10022c50     <common>
 0003:00001c54       __pDestructExceptionObject 10022c54     <common>
 0003:00001c58       ___piob                    10022c58     <common>
 0003:00001c60       __bufin                    10022c60     <common>
 0003:00002c60       __nstream                  10023c60     <common>
 0003:00002c64       __nhandle                  10023c64     <common>
 0003:00002c80       ___pioinfo                 10023c80     <common>
 0003:00002d80       ___env_initialized         10023d80     <common>
 0003:00002d84       ___onexitend               10023d84     <common>
 0003:00002d88       ___onexitbegin             10023d88     <common>
 0003:00002d8c       ___mbctype_initialized     10023d8c     <common>
 0003:00002d90       __FPinit                   10023d90     <common>
 0003:00002d94       ___dyn_tls_init_callback   10023d94     <common>
 0003:00002d98       __acmdln                   10023d98     <common>

 entry point at        0001:0000f575

 Static symbols

 0001:00000270       _adler32_combine_          10001270 f    CIL library: CIL module
 0001:00000450       _crc32_little              10001450 f    CIL library: CIL module
 0001:00000710       _gf2_matrix_times          10001710 f    CIL library: CIL module
 0001:00000730       _gf2_matrix_square         10001730 f    CIL library: CIL module
 0001:00000760       _crc32_combine_            10001760 f    CIL library: CIL module
 0001:00000ee0       _putShortMSB               10001ee0 f    CIL library: CIL module
 0001:00000f10       _flush_pending             10001f10 f    CIL library: CIL module
 0001:00001a30       _read_buf                  10002a30 f    CIL library: CIL module
 0001:00001aa0       _lm_init                   10002aa0 f    CIL library: CIL module
 0001:00001b30       _fill_window               10002b30 f    CIL library: CIL module
 0001:00001c80       _deflate_stored            10002c80 f    CIL library: CIL module
 0001:00001dc0       _deflate_fast              10002dc0 f    CIL library: CIL module
 0001:000020a0       _deflate_slow              100030a0 f    CIL library: CIL module
 0001:00002460       _deflate_rle               10003460 f    CIL library: CIL module
 0001:000026d0       _deflate_huff              100036d0 f    CIL library: CIL module
 0001:00002830       _gz_reset                  10003830 f    CIL library: CIL module
 0001:00002870       _gz_open                   10003870 f    CIL library: CIL module
 0001:00002f10       _gz_load                   10003f10 f    CIL library: CIL module
 0001:00002f80       _gz_avail                  10003f80 f    CIL library: CIL module
 0001:00002fc0       _gz_next4                  10003fc0 f    CIL library: CIL module
 0001:000030a0       _gz_head                   100040a0 f    CIL library: CIL module
 0001:000034e0       _gz_decomp                 100044e0 f    CIL library: CIL module
 0001:00003680       _gz_make                   10004680 f    CIL library: CIL module
 0001:00003700       _gz_skip                   10004700 f    CIL library: CIL module
 0001:00003b90       _gz_init                   10004b90 f    CIL library: CIL module
 0001:00003c70       _gz_comp                   10004c70 f    CIL library: CIL module
 0001:00003d50       _gz_zero                   10004d50 f    CIL library: CIL module
 0001:000042d0       _fixedtables               100052d0 f    CIL library: CIL module
 0001:00005330       _fixedtables               10006330 f    CIL library: CIL module
 0001:00005350       _updatewindow              10006350 f    CIL library: CIL module
 0001:00006b00       _syncsearch                10007b00 f    CIL library: CIL module
 0001:00007370       _fopen64_file_func         10008370 f    CIL library: CIL module
 0001:000073c0       _fread_file_func           100083c0 f    CIL library: CIL module
 0001:000073e0       _fwrite_file_func          100083e0 f    CIL library: CIL module
 0001:00007400       _ftell64_file_func         10008400 f    CIL library: CIL module
 0001:00007420       _fseek64_file_func         10008420 f    CIL library: CIL module
 0001:00007470       _fclose_file_func          10008470 f    CIL library: CIL module
 0001:00007490       _ferror_file_func          10008490 f    CIL library: CIL module
 0001:000074f0       _win32_translate_open_mode 100084f0 f    CIL library: CIL module
 0001:00007560       _win32_build_iowin         10008560 f    CIL library: CIL module
 0001:000079e0       _init_block                100089e0 f    CIL library: CIL module
 0001:00007a60       _pqdownheap                10008a60 f    CIL library: CIL module
 0001:00007b40       _gen_bitlen                10008b40 f    CIL library: CIL module
 0001:00007d40       _gen_codes                 10008d40 f    CIL library: CIL module
 0001:00007da0       _build_tree                10008da0 f    CIL library: CIL module
 0001:00007fa0       _scan_tree                 10008fa0 f    CIL library: CIL module
 0001:00008080       _send_tree                 10009080 f    CIL library: CIL module
 0001:00008600       _build_bl_tree             10009600 f    CIL library: CIL module
 0001:000086d0       _send_all_trees            100096d0 f    CIL library: CIL module
 0001:00008db0       _compress_block            10009db0 f    CIL library: CIL module
 0001:000091c0       _detect_data_type          1000a1c0 f    CIL library: CIL module
 0001:00009230       _bi_reverse                1000a230 f    CIL library: CIL module
 0001:00009250       _bi_flush                  1000a250 f    CIL library: CIL module
 0001:000092d0       _bi_windup                 1000a2d0 f    CIL library: CIL module
 0001:00009330       _copy_block                1000a330 f    CIL library: CIL module
 0001:00009470       _unz64local_getShort       1000a470 f    CIL library: CIL module
 0001:000094d0       _unz64local_getLong        1000a4d0 f    CIL library: CIL module
 0001:00009560       _unz64local_getLong64      1000a560 f    CIL library: CIL module
 0001:000096a0       _strcmpcasenosensitive_internal 1000a6a0 f    CIL library: CIL module
 0001:00009740       _unz64local_SearchCentralDir64 1000a740 f    CIL library: CIL module
 0001:000099d0       _unzOpenInternal           1000a9d0 f    CIL library: CIL module
 0001:00009f70       _unz64local_DosDateToTmuDate 1000af70 f    CIL library: CIL module
 0001:00009ff0       _unz64local_GetCurrentFileInfoInternal 1000aff0 f    CIL library: CIL module
 0001:0000a9d0       _unz64local_CheckCurrentFileCoherencyHeader 1000b9d0 f    CIL library: CIL module
 0001:0000b3d0       _decrypt_byte              1000c3d0 f    CIL library: CIL module
 0001:0000b3f0       _update_keys               1000c3f0 f    CIL library: CIL module
 0001:0000b430       _init_keys                 1000c430 f    CIL library: CIL module
 0001:0000b470       _crypthead                 1000c470 f    CIL library: CIL module
 0001:0000b580       _allocate_new_datablock    1000c580 f    CIL library: CIL module
 0001:0000b5b0       _free_datablock            1000c5b0 f    CIL library: CIL module
 0001:0000b5d0       _init_linkedlist           1000c5d0 f    CIL library: CIL module
 0001:0000b5e0       _free_linkedlist           1000c5e0 f    CIL library: CIL module
 0001:0000b600       _add_data_in_datablock     1000c600 f    CIL library: CIL module
 0001:0000b6b0       _zip64local_putValue       1000c6b0 f    CIL library: CIL module
 0001:0000b710       _zip64local_putValue_inmemory 1000c710 f    CIL library: CIL module
 0001:0000b750       _zip64local_TmzDateToDosDate 1000c750 f    CIL library: CIL module
 0001:0000b7a0       _zip64local_getByte        1000c7a0 f    CIL library: CIL module
 0001:0000b7a0       _unz64local_getByte        1000c7a0 f    CIL library: CIL module
 0001:0000b7e0       _zip64local_getShort       1000c7e0 f    CIL library: CIL module
 0001:0000b840       _zip64local_getLong        1000c840 f    CIL library: CIL module
 0001:0000b8d0       _zip64local_getLong64      1000c8d0 f    CIL library: CIL module
 0001:0000ba10       _zip64local_SearchCentralDir 1000ca10 f    CIL library: CIL module
 0001:0000ba10       _unz64local_SearchCentralDir 1000ca10 f    CIL library: CIL module
 0001:0000bbc0       _zip64local_SearchCentralDir64 1000cbc0 f    CIL library: CIL module
 0001:0000ce10       _zip64FlushWriteBuffer     1000de10 f    CIL library: CIL module
 0001:0000f47f       ___DllMainCRTStartup       1001047f f   LIBCMT:dllcrt0.obj
 0001:0000f783       _write_char                10010783 f   LIBCMT:output.obj
 0001:0000f7b6       _write_string              100107b6 f   LIBCMT:output.obj
 0001:0001072f       _doexit                    1001172f f   LIBCMT:crt0dat.obj
 0001:0001208f       _flsall                    1001308f f   LIBCMT:fflush.obj
 0001:000125d0       __unwind_handler4          100135d0 f   LIBCMT:exsup4.obj
 0001:00013804       _parse_cmdline             10014804 f   LIBCMT:stdargv.obj
 0001:00013de6       ?CPtoLCID@@YAHH@Z          10014de6 f   LIBCMT:mbctype.obj
 0001:00013e15       ?setSBCS@@YAXPAUthreadmbcinfostruct@@@Z 10014e15 f   LIBCMT:mbctype.obj
 0001:00013e79       ?setSBUpLow@@YAXPAUthreadmbcinfostruct@@@Z 10014e79 f   LIBCMT:mbctype.obj
 0001:000140ad       ?getSystemCP@@YAHH@Z       100150ad f   LIBCMT:mbctype.obj
 0001:00014d42       _siglookup                 10015d42 f   LIBCMT:winsig.obj
 0001:00014f47       __onexit_nolock            10015f47 f   LIBCMT:onexit.obj
 0001:00015cc0       __tsopen_nolock            10016cc0 f   LIBCMT:open.obj
 0001:00016930       __unwind_handler           10017930 f   LIBCMT:exsup.obj
 0001:00016d86       ?x_ismbbtype_l@@YAHPAUlocaleinfo_struct@@IHH@Z 10017d86 f   LIBCMT:ismbbyte.obj
 0001:00016e11       ?__crtLCMapStringA_stat@@YAHPAUlocaleinfo_struct@@KKPBDHPADHHH@Z 10017e11 f   LIBCMT:a_map.obj
 0001:0001703e       ?__crtGetStringTypeA_stat@@YAHPAUlocaleinfo_struct@@KPBDHPAGHHH@Z 1001803e f   LIBCMT:a_str.obj
